:100000000C94550E0C94720E0C94720E0C94720E8D
:100010000C94720E0C94720E0C94720E0C94720E60
:100020000C94720E0C94AF120C94720E0C94720E0F
:100030000C94720E0C94720E0C94720E0C94720E40
:100040000C94720E0C94AF0F0C943E2E0C94122E46
:100050000C94720E0C94720E0C94720E0C94720E20
:100060000C94720E0C94720E0C94720E0C94720E10
:100070000C94720E0C94720E0C94720E0C94720E00
:100080000C94720E0C94720E0C94720EF928892B3B
:100090000429892B202920297829BC29FB294B2ACE
:1000A0008D29892B892BE32AF42A1A2B2F2B892BB4
:1000B000892B892B892B892B892B892B892B892BA0
:1000C000892B892B892B6C2B6E2B732B402B892B27
:1000D000812B322E302E3100696E636F6D7061742A
:1000E00069626C6520485700202025303258002076
:1000F000504300204C430045617379436F6E747226
:100100006F6C000102031718040506151107080992
:1001100016120A000B0C13100F0E0D14040E1F0EF6
:100120000E0E0E000E0E0E0E1F0E0400040E1F000B
:100130001F0E0400000404040010081300100B1329
:1001400000130B130001021900011A1900191A19E2
:10015000080C1E1F1E0C080002060F1F0F060200CF
:100160000E11111F1B1B1F001F0A0A0A0A0A1F007B
:100170001C101810160505050C17141714170C0081
:10018000040A110A0A0E00001C10181216020207B7
:100190001C101816110204071C1018161102010673
:1001A0001C1018151507010100000017151515176B
:1001B000121212121200000000000017111714177B
:1001C0001711131117000000000000151517111169
:1001D0001714171117000000070505050505050789
:1001E0000707070707070707030509121418100078
:1001F00003070F1E1C18100000060912141209062E
:1002000000060917170906001F111F001F111F0004
:100210001F111F001F1F1F001F1F1F001F111F0086
:100220001F1F1F001F1F1F00040E1F04041F0E04AA
:10023000010101050D1F0C0411040A11111F110009
:10024000110E111111110E000A00111111110E00E1
:100250000E11111611111610001C1F1F1F13101064
:10026000001C13111D13101000181711191710106E
:10027000001F11111F101010206D332020200000CE
:10028000204D4D4920200000204D4D02202000002F
:1002900020444343202000002053544F50200000AE
:1002A00053484F52542100002048414C5420000034
:1002B00020202020202000002050524F4720000006
:1002C0005245534554200000202054504D2000003A
:1002D000555044415445000020202020002533641F
:1002E00000252D31312E31317300252D3564002547
:1002F000632F256320256300256300462530326483
:100300003D25630020200102202020202020200005
:100310002533640025336400252D3564002D2D2DF3
:100320002D2020004144523A20256C6420202020BA
:1003300020202020202000232D007E0E0E0E0E1BDC
:100340001B1C0E1B1B7E0E0E0E0E636F72746F2035
:1003500028312E356D73292000006C756E676F2073
:1003600028342E3032356D7329004D6F746F726FE3
:100370006C61000000000000000044434320202086
:10038000202000000000000000004D4D2000000073
:100390000000000000000000000044434300000093
:1003A00000000000000000000000706F73697469B5
:1003B000766120284D4D290000006E6567617469E3
:1003C00076612028444343290000303A206F666656
:1003D00020202020202020202000313A2054616954
:1003E0006C626974732020202000323A202B20494F
:1003F000644E6F74696679202000333A202B2041C7
:1004000063636573736F72792000526970726973E8
:1004100074696E6120202020200053616C76612079
:100420002020202020202020200052697072697333
:1004300074696E6120202020200053616C76612059
:100440002020202020202020200020737461746F41
:10045000206C61796F757420200020737461746F53
:10046000206C61796F7574202000636F72746F2047
:1004700028312E356D73292020006C6172676F2042
:1004800028342E3032356D7329004D6F746F726FC2
:100490006C61000000000000000044434320202065
:1004A000202000000000000000004D4D2000000052
:1004B0000000000000000000000044434300000072
:1004C00000000000000000000000706F7369746994
:1004D000766120284D4D290000006E6567617469C2
:1004E00076612028444343290000303A2044657354
:1004F000616374697661646F2000313A20546169E8
:100500006C626974732020202000323A202B20492D
:10051000644E6F74696679202000333A202B2041A5
:1005200063636573736F72792000526573746175CC
:100530007261722020202020200047756172646162
:1005400072202020202020202000526573746175C5
:100550007261722020202020200047756172646142
:100560007220202020202020200020457374616408
:100570006F204D617175657461002045737461640D
:100580006F204D617175657461004B75727A20281A
:10059000312E356D7329202000004C616E672028B4
:1005A000342E3032356D732900004D6F746F726FC9
:1005B0006C61000000000000000044434320202044
:1005C000202000000000000000004D4D2000000031
:1005D0000000000000000000000044434300000051
:1005E00000000000000000000000706F7369746973
:1005F0007620284D4D29000000006E656761746902
:1006000076202844434329000000303A2061757366
:1006100020202020202020202000313A2054616911
:100620006C626974732020202000323A202B20490C
:10063000644E6F74696679202000333A202B204184
:1006400063636573736F72792000416E6C616765D7
:100650006E7A757374616E642000416E6C616765BB
:100660006E7A757374616E64200057696564657293
:100670006865727374656C6C6E005370656963684D
:1006800065726E2020202020200020776965646537
:100690007268657273742E20200020737065696320
:1006A0006865726E20202020200073686F727420AD
:1006B00028312E356D73292000006C6F6E6720285D
:1006C000342E3032356D732900004D6F746F726FA8
:1006D0006C61000000000000000044434320202023
:1006E000202000000000000000004D4D2000000010
:1006F0000000000000000000000044434300000030
:1007000000000000000000000000706F7369746951
:10071000766520284D4D290000006E65676174697B
:1007200076652028444343290000303A206F6666EE
:1007300020202020202020202000313A20546169F0
:100740006C626974732020202000323A202B2049EB
:10075000644E6F74696679202000333A202B204163
:1007600063636573736F72792000526573746F727F
:100770006520202020202020200053617665202045
:1007800020202020202020202000526573746F72CA
:100790006520202020202020200053617665202025
:1007A00020202020202020202000206C61796F75DF
:1007B00074207374617475732000206C61796F7597
:1007C000742073746174757320005B756E6B6E6F4B
:1007D000776E207374617475735D00466F726D611E
:1007E000746F20696E636F6D70617400466F726D17
:1007F00061746F20696E636F6D702E2000696E6B7F
:100800006F6D7061742E20466F726D617400696E39
:10081000636F6D7061742E20466F726D6174005B42
:10082000756E6B6E6F776E206572726F725D002EE3
:100830002E20617474656E64657265202E2E200012
:10084000233D63616E63656C6C6100000000000015
:10085000002876756F746F2900000000000000000A
:1008600000002E2E63616E63656C6C617A696F6E39
:10087000652E00206572726F726500000000000036
:100880000000000020736F6C6F2044434321202040
:100890002020202000207072696D61207072656DCB
:1008A0006920474F20002A3D416E6E756C6C6100D7
:1008B000000000000000002070726F6772616D6DB3
:1008C000617A696F6E6520002D636F72746F2063AB
:1008D0006972637569746F2D00206E617469766F3B
:1008E0002028313A312920202000206C696E656172
:1008F00072652028323A31292020002070726F67FB
:100900007265737369766F20312020002070726FDA
:10091000677265737369766F2032202000204D6FF7
:10092000646F204143202020202020202000204DE3
:100930006F646F20444320202020202020200020AE
:100940004175746F53746570202020202020200092
:100950002A6C656767692000000000000000000045
:10096000002A7363726976690000000000000000CD
:1009700000002E2E20736372697474757261202ECC
:100980002E20002E2E2E206C657474757261202E20
:100990002E2E2000212121206572726F7265202188
:1009A0002121202000204F4B20202020202020200B
:1009B0002020202020002E2073616C7661746167F6
:1009C00067696F202E20002E2E2072697072697365
:1009D00074696E6F202E2000233D43616E63202AD0
:1009E0003D416E6E756C202000233D5369202A3DE9
:1009F000416E6E756C6C6120200020636F6E6669BD
:100A0000677572617A696F6E6520005350454E5468
:100A10004F00000000000000000000002A204E658A
:100A20007373756E205472656E6F202A0020636F99
:100A300072746F20636972637569746F20002A2A6B
:100A40002A2074696D65206F7574202A2A2A004156
:100A500063636573732E20202534642F253464006E
:100A6000436F6E6669677572617A696F6E65202083
:100A70000020636F6E6669677572617A696F6E6573
:100A800020002E2E2E20657370657265202E2E2E6E
:100A9000202000233D626F7272617200000000002E
:100AA000000000002873696E2046696368612900B0
:100AB00000000000002E2E2E20626F7272616E64A4
:100AC0006F202E2E2E002046616C6C6F00000000FF
:100AD0000000000000000020736F6C6F20706172D6
:100AE00061204443432120002022474F222070727E
:100AF000696D65726F202020002A3D43616E636539
:100B00006C6172000000000000002050726F67727C
:100B1000616D6163696F6E202020002D636F7274B8
:100B20006F20636972637569746F2D00206E617444
:100B300069766F2028313A312920202000206C6905
:100B40006E6561722028323A312920202000207001
:100B5000726F677265737369766F20312020002091
:100B600070726F677265737369766F203220200030
:100B7000204D6F646F204143202020202020202022
:100B800000204D6F646F204443202020202020202F
:100B90002000204175746F53746570202020202040
:100BA0002020002A6C656572200000000000000013
:100BB000000000002A6573637269000000000000F5
:100BC00000000000002E2065736372696269656E23
:100BD000646F202E20002E2E2E206C6579656E64A9
:100BE0006F202E2E2E20002121212046616C6C6F5B
:100BF0002021212120202000204F4B2020202020B8
:100C00002020202020202020002E2E2067756172B9
:100C100064616E646F202E2E20002E207265737426
:100C2000617572616E646F202E2000233D426F72E9
:100C30007261202A3D43616E632E2000233D53697B
:100C4000202A3D43616E63656C6172200020436F12
:100C50006E66696775726163696F6E202000446516
:100C60007361637469766164612020202020002A0A
:100C70002A2A2053696E205472656E202A2A2A007F
:100C80002A636F72746F20636972637569746F2A67
:100C9000005469656D706F20657870697261646F6A
:100CA000200041636365732E202534642F2534644E
:100CB000000000436F6E66696775726163696F6EED
:100CC0002020200020436F6E66696775726163693A
:100CD0006F6E2020002E2E2E2077617274656E209C
:100CE0002E2E2E202000233D4CF6736368656E0087
:100CF00000000000000000286B65696E2045696EE9
:100D00007472616729000000202E2E2E206CF6736D
:100D1000636865202E2E2E2000204665686C657263
:100D200000000000000000000000206E75722066C8
:100D3000FC722044434321202020002065727374FC
:100D400020474F206472FC636B656E002A3D416250
:100D5000627275636800000000000000002050729D
:100D60006F6772616D6D696572756E6700002D2D1C
:100D7000204B75727A7363686C75DF202D2D00200F
:100D80004E617469762028313A31292020202000D4
:100D9000204C696E6561722028323A31292020206A
:100DA000002050726F67726573736976203120205E
:100DB00020002050726F677265737369762032204D
:100DC000202000204143204D6F6475732020202097
:100DD00020202000204443204D6F64757320202084
:100DE0002020202000204175746F537465702020EE
:100DF0002020202020002A6C6573656E0000000012
:100E0000000000000000002A736368722E000000DA
:100E100000000000000000002E2E20736368726541
:100E20006962656E202E2E00002E2E2E206C6573BA
:100E3000656E202E2E2E20200000212121204665C7
:100E4000686C657220212121200000204F4B20205A
:100E50002020202020202020202000002E2E207363
:100E6000706569636865726E202E2E000077696573
:100E70006465726865727374656C6C656E00233DA1
:100E80004CF6736368656E202A3D416262720023EE
:100E90003D4A61202A3D416262727563680000002C
:100EA000206CF6736368656E2020202020202020AF
:100EB0000041555300000000000000000000000049
:100EC00000002A2A206B65696E65204C6F6B202A12
:100ED0002A20002A2A204B75727A7363686C75DFAA
:100EE000202A2A002A205A656974FC62657273639D
:100EF00068722E2A00576569636865202534642F5F
:100F00002534640000004B6F6E666967757261740A
:100F1000696F6E20202000204B6F6E6669677572C6
:100F20006174696F6E2020002E2E2E207761697407
:100F3000696E67202E2E2E2000233D64656C65743B
:100F400065000000000000000000286E6F20656E44
:100F500074727929000000000000002E2E2E2064FB
:100F6000656C6574696E67202E2E2E002066617593
:100F70006C740000000000000000000000204443EA
:100F800043206F6E6C7921202020202020002070CB
:100F90007265737320474F20666972737400002A6C
:100FA0003D43616E63656C000000000000000000BE
:100FB0002070726F6772616D696E670000000000DB
:100FC000002D73686F727420636972637569742D84
:100FD0002000206E61746976652028313A3129201D
:100FE000202000206C696E6561722028323A312918
:100FF000202020002070726F6772657373697665B8
:1010000020312020002070726F67726573736976DB
:10101000652032202000204143204D6F6465202050
:1010200020202020202000204443204D6F64652094
:101030002020202020202000204175746F537465EB
:101040007020202020202020002A7265616420006A
:10105000000000000000000000002A77726974653B
:1010600000000000000000000000002E2E2E20775F
:10107000726974696E67202E2E2E20002E2E2E206F
:1010800072656164696E67202E2E2E200021212159
:10109000206661756C742021212120202000204FC2
:1010A0004B20202020202020202020202020002E27
:1010B0002E2E20736176696E67202E2E2E20200042
:1010C0002E2E20726573746F72696E67202E2E202B
:1010D00000233D44656C2E202A3D43616E63656CA0
:1010E0002000233D596573202A3D43616E63656C82
:1010F00020200020636F6E66696775726174696F86
:101100006E2020004F464600000000000000000056
:1011100000000000002A2A2A206E6F2054726169A4
:101120006E202A2A2A002A2073686F72742063694D
:10113000726375697420002A2A2A2074696D6520FB
:101140006F7574202A2A2A00506F696E742020253A
:1011500034642F253464000000436F6E6669677540
:10116000726174696F6E2020200020636F6E666963
:101170006775726174696F6E2020005B6E6F206D01
:101180006573736167655D004003A001CF00670070
:101190004400330019001000204D3320656E616259
:1011A0006C65642020202020003D253564003078C7
:1011B0002530386C580020253564002534646D7363
:1011C000002533642C25647300202E2E2E2E202023
:1011D00020202020202020002564206D7300202561
:1011E00032640025346400202D2D2D002020202085
:1011F00020202000204F4B20202020002533640099
:101200002D2D2D002534643A200025366400202D34
:101210002D2D2D2D0025346400202D2D2D0043561D
:101220003A253464204269743A25643D0043563AB5
:1012300020202020204269743A203D200025357569
:1012400000202D2D2D2D004142434445464748495D
:101250004A4B4C4D4E4F5051525354555657585976
:101260005A303132333435363738392E2C3A2D2B2B
:10127000232F3D3C7C3E20004D4D20492020313421
:1012800020004D4D20492020323761004D4D20492E
:101290002020323762004D4D2002202031342000C2
:1012A0004D4D20022020323761004D4D200220207C
:1012B000323762004443432020203134200044432D
:1012C000432020203238200044434320203132384C
:1012D00020006D3320202031323820003A200025B4
:1012E0003575005365724E722E2025386C750032AC
:1012F0002E302E3100536F6674772E205600253322
:1013000064004E723A202532642020004D656E75CF
:10131000204C6F636F6D6F746976650050726F67F4
:1013200072616D6D617A2E204443430050726F6785
:1013300072616D6D617A2E206D330000537461749B
:101340006F204C61796F757400000000496D706FFB
:1013500073746174696F6E65000000004C43442033
:10136000726574726F696C6C2E0000004C6F6B4379
:101370006F6E74726F6C000000000000557363693B
:1013800074610000000000000000000053656C65FF
:101390007A696F6E6120000000000000466F726D78
:1013A00061746F2044617469200000004E6F6D65A8
:1013B00020202020202000000000000056616C6FDB
:1013C00072652020202020000000000043562028C5
:1013D000627974652900000000000000435620284F
:1013E000626974290000000000000000496E642E4C
:1013F000205072696D6172696F000000496E642E41
:101400002045737465736F000000000052656769C2
:101410007374726F00000000000000005061676587
:101420002D4D6F6465000000000000004D61696E85
:1014300020547261636B0000000000005261696C0F
:10144000436F6D2043560000000000004D6F646F35
:101450002031323846530000000000004D6F646FA9
:10146000204A6F676469616C00000000496D706F0D
:101470007374617A2E2073383800000043616E6304
:10148000656C6C610000000000000000426F6F732B
:1014900074657200000000000000000056656C6F6B
:1014A0006369746120696E74657266004465632EB9
:1014B0004163636573736F7269000000466F726DFC
:1014C00061746F204C6F636F000000005061757392
:1014D00061207365676E2E4D4D200000537570704E
:1014E0006F72742E5261696C436F6D006D6F64751D
:1014F0006C69207338380000000000007465737454
:10150000206D6F64756C692073383800506F6C2ED5
:1015100020636F72746F636972632E0053656E731C
:101520002E20636F72746F6369722E005475747429
:1015300069206163636573736F726900466F726DD2
:101540002E206163636573736F7269006D696E2E1F
:10155000746D702E696D70756C736F006D61782E8F
:10156000746D702E696D70756C736F00696E64694F
:1015700072697A7A6F206D33000000004D656E75D8
:10158000204C6F636F6D6F746F72610050726F6784
:1015900072616D6D617220444343000050726F6749
:1015A00072616D6D6172206D33000000457374616E
:1015B000646F204D6171756574610000416A7573D7
:1015C000746573000000000000000000496C756D38
:1015D000696E6163696F6E204C4344004C6F6B43CE
:1015E0006F6E74726F6C00000000000053616C69D4
:1015F00072000000000000000000000053656C65F0
:101600006363696F6E61722000000000466F726D47
:1016100061746F204461746F730000004E6F6D62DF
:1016200072652020202000000000000046696368E9
:1016300061202020202000000000000043562028C8
:1016400062797465290000000000000043562028DC
:10165000626974290000000000000000446972659E
:101660006363696F6E20636F7274610044697265B1
:101670006363696F6E206C617267610052656769B0
:101680007374726F00000000000000005061676515
:101690002D4D6F646500000000000000456E20566F
:1016A0006961207072696E6369702E005261696CA5
:1016B000436F6D2043560000000000004D6F646FC3
:1016C00020313238207061736F7300004D6F646F8A
:1016D000206465206D616E646F000000416A75735F
:1016E000746573207338380000000000426F727216
:1016F000617200000000000000000000426F6F7384
:101700007465723A000000000000000041636365E8
:10171000736F72696F733A0000000000466F726D5C
:1017200061746F206465205472656E00506175733A
:1017300061205365F1616C204D4D00005375706F51
:10174000727465205261696C436F6D004D6F6475F2
:101750006C6F73207338380000000000507275659C
:101760006261204D6F642E2073383800506F6C2EEC
:1017700020436F72746F636972632E0053656E73DA
:101780002E20436F72746F6369726300546F646FCD
:10179000732041636365736F722E0000466F726D34
:1017A00061746F2061636365736F72004475726169
:1017B000632E496D70756C2E6D696E004475726193
:1017C000632E496D70756C2E6D6178004469726589
:1017D0006363696F6E206D33000000004C6F6B20F7
:1017E0004D656EFC00000000000000004443432DE6
:1017F00050726F6772616D6D672E00006D332050FF
:10180000726F6772616D6D672E000000416E6C61D2
:1018100067656E7A757374616E64000045696E73F6
:1018200074656C6C756E67656E0000004C434420F7
:1018300042656C6575636874756E67004C6F6B43C9
:101840006F6E74726F6C0000000000004578697460
:1018500000000000000000000000000041757377E8
:10186000E4686C656E20000000000000446174654F
:101870006E666F726D617400000000004E616D65F0
:1018800020202020202000000000000045696E7408
:1018900072616720202000000000000043562028CD
:1018A000627974652900000000000000435620287A
:1018B0006269742900000000000000004261736941
:1018C000732D416472657373650000006C616E670F
:1018D0006520416472657373650000005265676935
:1018E00073746572000000000000000050616765BD
:1018F0002D4D6F64650000000000000048617570A8
:1019000074676C6569730000000000005261696CC7
:10191000436F6D204356000000000000313238460E
:1019200053204D6F64650000000000005265676C35
:1019300065726D6F64757300000000007338382D98
:1019400045696E7374656C6C756E67004B6F6E667F
:10195000696775726174696F6E000000426F6F7322
:1019600074657200000000000000000057656963A4
:1019700068656E0000000000000000004C6F6B66A0
:101980006F726D6174000000000000004D4D2D531A
:1019900069676E616C205061757365005261696C96
:1019A000436F6D20537570706F7274007338382DEB
:1019B0004D6F64756C650000000000007338382DB1
:1019C0004D6F64756C746573740000004B75727AAA
:1019D0007363686C2E2D506F6C2E00004B75727AFD
:1019E0007363686C2E2D456D70662E00616C6C659E
:1019F000205765696368656E00000000576569637C
:101A000068656E666F726D61740000006D696E2EA0
:101A100020536368616C747A656974006D61782E17
:101A200020536368616C747A656974006D3320417A
:101A30006472657373650000000000004C6F636F93
:101A40006D6F74697665206D656E75004443432043
:101A500070726F6772616D6D696E67006D332070B3
:101A6000726F6772616D6D696E6700004C61796FAE
:101A70007574207374617475730000005365747419
:101A8000696E677300000000000000004C434420B2
:101A90006261636B6C696768740000004C6F6B4334
:101AA0006F6E74726F6C00000000000045786974FE
:101AB00000000000000000000000000053656C659D
:101AC00063742000000000000000000044617461A5
:101AD00020666F726D617400000000004E616D65DC
:101AE000202020202020000000000000456E74729D
:101AF00079202020202000000000000043562028EC
:101B00006279746529000000000000004356202817
:101B10006269742900000000000000005072696DC5
:101B200061727920616464726573730045787465CD
:101B30006E642E2061646472657373005265676918
:101B4000737465720000000000000000506167655A
:101B50002D4D6F6465000000000000004D61696E4E
:101B600020747261636B0000000000005261696CB8
:101B7000436F6D20435600000000000031323846AC
:101B800053204D6F64650000000000004A6F6764D9
:101B900069616C204D6F6465000000007338382067
:101BA00073657474696E67730000000044656C654A
:101BB000746500000000000000000000426F6F73B9
:101BC000746572000000000000000000506F696E34
:101BD0007473000000000000000000004C6F632ED2
:101BE00020666F726D617400000000004D4D20731F
:101BF00069676E616C207061757365005261696C14
:101C0000436F6D20537570706F7274007338382095
:101C10006D6F64756C6573000000000073383820C8
:101C20006D6F64756C6520746573740053686F72B2
:101C30007420632E20706F6C2E00000053686F724A
:101C40007420632E2073656E732E0000616C6C200F
:101C5000506F696E7473000000000000506F696E71
:101C6000747320666F726D61740000006D696E2E72
:101C70007377697463682E74696D65006D61782E81
:101C80007377697463682E74696D65006D332061C4
:101C9000646472657373000000000000202020302F
:101CA000782530386C582020200011241FBECFEF3B
:101CB000D0E1DEBFCDBF11E0A0E0B1E0ECE8FEE98D
:101CC00002C005900D92A23DB107D9F714E0A2ED34
:101CD000B1E001C01D92A238B107E1F70E94920E57
:101CE0000C94444F0C9400008091D201089581E03F
:101CF0008093D301089580E00E94ED16BC018FEF20
:101D00006F3F780719F080E00E94EC2F0E948D272A
:101D10000E94C4198091D301882311F40E9489156F
:101D2000A8950895CF93DF930E945C260E946E0FC2
:101D300083E068E04EE422E00E94D02D0E9438113A
:101D400078940E9461130E943725DC0114968C91CF
:101D50000E94841582E067EF70E00E94CF170E9416
:101D60004B25823021F00E944B25813021F482E006
:101D700063EF70E007C00E944B258038D9F482E001
:101D80006FEE70E00E94CF1781E060E00E940716BE
:101D900082E066E50E94FC1682E062ED70E00E943F
:101DA000CF170E943725EC0181E00E943714882369
:101DB00049F125C00E944B2500D000D00F92EDB70D
:101DC000FEB7319692E0ADB7BEB711969C9328EE60
:101DD00030E032832183838314820E9475170F9031
:101DE0000F900F900F900F9081E060E00E94071617
:101DF00082E068ED70E00E94CF17A895FECF80E0EA
:101E00000E94432682E00E943714882319F084E060
:101E10000E94432683E00E943714882319F085E04E
:101E20000E94432684E00E943714882329F081E031
:101E30000E94432601C0A8950E94DA278823D9F37F
:101E400089859A85009749F060E070E040E050E0B5
:101E50000E94392DBC01009711F46A817B818FEFBC
:101E60000E94EF2581E011C00E9441200E945B1476
:101E7000BFEF8F3F9B07C1F70E947B0E8091D3017C
:101E80008823A1F31092D30180E00E944A1BEECF79
:101E90009091D201981701F19630F1F0953011F43C
:101EA0008630D1F48093D201853029F480E060E25D
:101EB00045E00E940A278091D201863029F480E013
:101EC00060E246E00E940A278091D2010E94AF2F73
:101ED00081E08093D301089580E008958FE78ABB65
:101EE0001BBA80E187BB18BA80EF84BB8FEF85BB3C
:101EF0008BEB81BB8CEC82BB82E082B987EF83B92C
:101F000087E78093610081EE8093620087E1809390
:101F1000640089E1809365000E941A12A89588E107
:101F200081BD8EE081BD0895DC019091D70189E0EB
:101F3000989FF0011124EF52FC4F90E08D91819316
:101F40009F5F9930D9F78091D7018F5F8093D70138
:101F50008091D701843010F01092D70108951F921C
:101F60000F920FB60F9211241F932F933F934F930D
:101F70005F936F937F938F939F93AF93BF93EF93F1
:101F8000FF9380910001909101012FEF8F3F920705
:101F900061F0BB9A8FB9769B0BC0BB981092D601AB
:101FA0001092DC011092DB0103C0BB988FEF8FB958
:101FB0001FB117FF8AC08091DD019091DE01892B4E
:101FC000E1F08091D9018F5F8093D9018091D9018F
:101FD000803210F01092D9019091D9018091DA01EC
:101FE000981759F48091DA018F5F8093DA0180911C
:101FF000DA01803210F01092DA018091DB019091C9
:10200000DC01815D934061F058F08091D8018F5FD1
:102010008093D8018091D801843010F01092D801BB
:102020001092DE011092DD011092DC011092DB01B2
:1020300080910201181721F481E08093D60177C0C6
:102040001092D601412F50E04F775070682F70E00A
:102050004617570729F01F3F19F08F3F09F067C057
:102060008091D90129E0829FC00111248F549D4F96
:102070009093DE018093DD014617570709F057C0A2
:102080009091D7018091D801981721F488EA92E0C5
:102090000E94940F8091D80129E0829FC0011124F1
:1020A0008F529C4F9093DC018093DB018091D8018B
:1020B0008F5F8093D8018091D801843010F0109206
:1020C000D80189E08093D40132C02091D60121301B
:1020D00029F0213060F1263050F515C082E0809360
:1020E000D601103419F41092D50121C0113419F41D
:1020F0002093D5011CC0123419F0133491F483E0FD
:102100008093D50114C0E22FF0E08091D50190E0DA
:1021100002968E179F0744F0E352FE4F80811817F6
:1021200019F01092D60103C02F5F2093D601809141
:10213000D601882329F0109300011092010121C0DB
:10214000E091DB01F091DC013097A9F0819180935F
:10215000000110920101F093DC01E093DB0180911A
:10216000D40181508093D401882359F41092DC016A
:102170001092DB0106C08FEF9FEF909301018093D7
:102180000001E091DD01F091DE01309749F083E03C
:10219000E13DF80728F41193F093DE01E093DD01AF
:1021A000FF91EF91BF91AF919F918F917F916F912F
:1021B0005F914F913F912F911F910F900FBE0F9004
:1021C0001F9018951F93AC011FB7F8942091D70169
:1021D0008091D80130E090E001972817390741F04D
:1021E0008091D701833039F48091D801882319F484
:1021F0001FBF80E005C0CA010E94940F1FBF81E08D
:102200001F910895DC01E8EAF2E08D91819382E06C
:10221000E13BF807D1F708959C01009739F14FB7DA
:10222000F8949091D9018091DA01981721F44FBF69
:1022300020E030E01BC09091DA0189E0989FF00126
:102240001124EF54FD4FD90190E081918D939F5F50
:102250009930D9F78091DA018F5F8093DA0180910C
:10226000DA01803210F01092DA014FBFC9010895EF
:102270000E944125262F2F772093E20147E0969573
:102280008795779567954A95D1F7262F2F772093D5
:10229000E10137E096958795779567953A95D1F75F
:1022A000262F2F772093E00127E096958795779545
:1022B00067952A95D1F76F776093DF0187B3807FA9
:1022C00087BB88B3807F88BB84EE8DB9089588234F
:1022D00051F08091650084608093650000000000EB
:1022E000000000000895809165008B7F8093650059
:1022F00008950F931F93DF93CF930F92CDB7DEB75F
:10230000182F8AB3807F8ABB80E00E94671180917A
:102310006500826080936500112321F08091650043
:10232000816003C0809165008E7F8093650000000E
:10233000000081E00E94671109B380E00E946711EC
:1023400010E084E0000F111F8A95E1F70000000003
:102350000000000081E00E94671199B39F70902BEC
:1023600080E099830E9467118AB38F608ABB99814C
:10237000892F0F90CF91DF911F910F91089580E0E9
:102380000E947911982F87FF11C08091E6019091EA
:10239000E70128E08130920714F080E0089501966B
:1023A0009093E7018093E60181E008958091E80130
:1023B000882319F49F779093E9011092E701109216
:1023C000E60180E008959B01AC018091F7039091B4
:1023D000F803A091F903B091FA0382179307A407B9
:1023E000B50798F08091F7039091F803A091F90355
:1023F000B091FA0360E0821B930BA40BB50B8050E5
:102400009041A040B040A0F412C08091F703909199
:10241000F803A091F903B091FA0360E0281B390B8F
:102420004A0B5B0B2050304F4F4F5F4F08F061E07D
:10243000862F089510927D0080B7877F80BF17BEDA
:1024400011BE89E683BF8BE085BD8FE183BD87B771
:10245000806887BF0895EF92FF920F931F9320919A
:10246000F7033091F8034091F9035091FA037C018E
:1024700000E010E0E20EF31E041F151F01C0A89536
:10248000C801B7010E94E3118823C9F31F910F917E
:10249000FF90EF900895FF920F931F93082F162F30
:1024A000F42E809165008D7F8093650080E00E940E
:1024B00067118AB38F608ABB8BB3902F92959F7000
:1024C000807F982B9BBB112321F080916500816058
:1024D00003C0809165008E7F8093650081E00E943B
:1024E000671180E00E946711FF2029F088E090E0EA
:1024F0000E942B120FC08BB30F70807F802B8BBB81
:10250000000000000000000081E00E94671180E0F0
:102510000E9467111F910F91FF900895EF92FF9213
:102520000F931F932091F7033091F8034091F90323
:102530005091FA037C0100E010E0E20EF31E041F4C
:10254000151F02C00E947B0EC801B7010E94E31153
:102550008823C1F31F910F91FF90EF9008951F9270
:102560000F920FB60F9211241F932F933F934F9307
:102570005F936F937F938F939F93AF93BF93EF93EB
:10258000FF938091E301882309F089C081E0809363
:10259000E30178948091E5018F5F8093E50180915C
:1025A000E50190E083709070009719F0019741F574
:1025B00016C08091F7039091F803A091F903B091B0
:1025C000FA030196A11DB11D8093F7039093F803C0
:1025D000A093F903B093FA030E94431411C08091B1
:1025E000F7039091F803A091F903B091FA03817079
:1025F0009070892B19F00E94751402C00E94FB1381
:102600008091E401882321F00E94BF118093E401AE
:102610008091E401882309F040C09091FB038091F0
:10262000FC039817B9F18091FC03E82FF0E0E55026
:10263000FC4F9281182F1F5F103108F010E0903886
:1026400001F58091FB03811729F1E12FF0E0E550BE
:10265000FC4F92819F3F19F49091E901906897FF98
:1026600002C01092E801892F807C803419F481E047
:102670008093E8011F5F103108F010E0892F60E0BF
:1026800002C0892F61E040E00E944B121093FC03CE
:1026900081E001C080E08093E4011092E301FF91AA
:1026A000EF91BF91AF919F918F917F916F915F91CA
:1026B0004F913F912F911F910F900FBE0F901F9040
:1026C0001895CF93DF9388E290E00E942B1280E36D
:1026D00060E041E00E944B1280E360E041E00E9434
:1026E0004B1280E360E041E00E944B1280E260E028
:1026F00041E00E944B1288E20E94F11580E40E94A2
:10270000F1158AE00E94C41589E20E94F1158CE15E
:102710000E94F11582E50E94F11589E60E94F115EB
:1027200084E70E94F11580E40E94F11585E10E9482
:10273000C41588E20E94F11580E40E94F1150E9400
:10274000F817EC0101C0A8959091FB038091FC0360
:102750009817C9F70E94BF118823A9F781E00E944A
:1027600079118A3019F481E089AB01C019AA88E097
:102770000E94F11581E00E94F11586E00E94F1159A
:102780008CE00E94F11580E060E00E94071680E076
:102790006CE171E00E94E81681E060E671E00E9461
:1027A000E81682E068E671E00E94E81683E068E7D8
:1027B00071E00E94E816DF91CF9108959091EC01AD
:1027C000E92FF0E0E451FE4F82839F5F9093EC018C
:1027D000983010F01092EC019091ED018091EC0195
:1027E000981741F4892F8F5F8093ED01883010F0A6
:1027F0001092ED01089531B12091EB01220F36FDC9
:102800002160822F83708150823028F424FF02C01F
:102810002E6001C0217F2093EB019091EA01990F76
:1028200037FD9160892F83708150823028F494FFA6
:1028300002C09E6001C0917F9093EA01207C892FA5
:10284000807C203831F4882341F0803C79F48AE19F
:1028500005C0203459F4803C21F489E10E94DE1344
:102860000895882319F48AE10E94DE1308958931BE
:1028700010F080E00895E82FF0E0EA50FE4F8081EC
:10288000811181E0089530912802343029F485B314
:10289000806F85BB97980895979A25B380E190E063
:1028A00002C0880F991F3A95E2F78095807F2F70BC
:1028B000822B85BB08959091ED018091EC018917E1
:1028C00019F42FEF3FEF0FC0E92FF0E0E451FE4F76
:1028D0008281282F30E0892F8F5F8093ED0188302F
:1028E00010F01092ED01C90108958F929F92AF925E
:1028F000BF92CF92DF92EF92FF920F931F93CF93ED
:10290000DF930E94740E982F80912902981729F066
:102910009093290282E20E94DE1383B3E1B0EE0CB1
:10292000EE0C90E1E9228F70E82ACC24DD2495E0BA
:10293000892E81E0A82EB12C99249394E09128024D
:10294000E89DF0011124EC0DFD1DED5FFE4FF490AC
:1029500088E18F1508F481C00E2D0A250170CF2D56
:10296000D0E0FE01E15FFD4F1081110F0E944B2569
:10297000803819F4002371F009C001111160812F12
:1029800090E0817190708131910511F41F6103C055
:10299000892B09F4107E812F90E08076907080342E
:1029A000910519F41F7182E00CC08032910519F471
:1029B000106E81E006C08036910511F080E001C004
:1029C00083E0FE01E15FFD4F1083823099F0833098
:1029D00059F1813009F041C096E1F91621F4809156
:1029E0000B02882319F48F2D0E94DE13CA50DE4F8C
:1029F000988233C0CA50DE4F18828F2D80680E94A3
:102A0000DE130E94740E853041F585E1F81619F445
:102A100080910C0205C096E1F916F9F480910B0241
:102A20008823D9F486E017C0FE01EA50FE4F80816A
:102A30008F5F8083882309F490828BEEF80E91E0FB
:102A40009F1558F080910B02893738F080910C0265
:102A5000893718F085E00E94480F0894C11CD11CEA
:102A600085E0C816D10411F0E69468CF8091280261
:102A70008F5F80932802853010F010922802DF913A
:102A8000CF911F910F91FF90EF90DF90CF90BF906B
:102A9000AF909F908F90089590932804809327047F
:102AA000892B89F170932604609325048091F703A4
:102AB0009091F803A091F903B091FA039B0140E0D3
:102AC00050E0280F391F4A1F5B1F209321043093C9
:102AD00022044093230450932404809120048E7F89
:102AE00080932004211531054105510561F481E0F1
:102AF00090E0A0E0B0E08093210490932204A093A2
:102B00002304B09324040895813308F080E381BF47
:102B100008958091270490912804892BA1F1609158
:102B200021047091220480912304909124040E9436
:102B3000E311882341F180912004E0912704F09172
:102B40002804817009958091200491E08927809361
:102B500020042091F7033091F8034091F90350913C
:102B6000FA038091250490912604A0E0B0E0820F42
:102B7000931FA41FB51F8093210490932204A09358
:102B80002304B093240408951F93182F03C00E94B8
:102B90008D27A8952091FB038091FC0330E090E005
:102BA00001972817390799F38091FB038F3021F49F
:102BB0008091FC03882359F3F894E091FB03F0E043
:102BC000E550FC4F12838091FB038F5F8093FB03E2
:102BD0008091FB03803110F01092FB0378941F91D9
:102BE00008951F93182F80E80E94C415812F0E941A
:102BF000C4151F910895109228041092270481E0B3
:102C00000E94F11508958CE00E94F11508958295B7
:102C1000880F880F807C860F80680E94F1150895C8
:102C2000BF92CF92DF92EF92FF920F931F93CF93B9
:102C3000DF93C82EB62E8A01109228041092270422
:102C400021E02817A0F13FE0361788F14115510522
:102C500071F1FA0101900020E9F73197DE2ED41AC4
:102C600080E18D1510F490E1D92E8C2D6B2D0E94F2
:102C70000716E8018DE0E82E84E0F82E08C0888170
:102C8000F70181937F01699182E00E94FC169E0109
:102C9000201B2D15A0F3C0921D04B0921E04D092EB
:102CA0001F048AE896E164EF71E00E944C15DF9101
:102CB000CF911F910F91FF90EF90DF90CF90BF9039
:102CC0000895DF93CF93CDB7DEB7A0970FB6F894F2
:102CD000DEBF0FBECDBFDE0111969E01205E3F4FCD
:102CE00004C09D93A217B30731F0FA014F5F5F4F05
:102CF00094919923B1F71C92AE014F5F5F4F0E94F0
:102D00001016A0960FB6F894DEBF0FBECDBFCF91C0
:102D1000DF9108950F931F93CF93DF93082F809136
:102D20001D0460911E040E94071610E0CDE0D4E05F
:102D300009C0002311F460E201C0699182E00E94A1
:102D4000FC161F5F80911F04181798F3DF91CF9135
:102D50001F910F9108950E9407168EE00E94F115B1
:102D60000895EF92FF920F931F93CF93DF93382F25
:102D70007B01122F883028F5483018F5842F90E019
:102D8000820F911D099714F018E0141B330F330FB5
:102D9000330F340F832F80640E94F115C0E0D0E020
:102DA000012F10E008C0F701EC0FFD1FE4918E2FFA
:102DB0000E94C4152196C017D107ACF38FEF0E9473
:102DC000F115DF91CF911F910F91FF90EF90089532
:102DD00040E028E00E94B1160895882341F0833036
:102DE00019F02FEF3FEF06C00E945B1402C00E9453
:102DF0003A2F9C01C90108951F93162F882309F4C7
:102E00005EC0823009F05EC067FF55C00E94F817AF
:102E1000FC0181A98823E1F0143E11F414E84BC0B1
:102E2000163F11F414E947C01C3F11F411E843C0E8
:102E3000143C11F41EE83FC0163D11F419E93BC0E3
:102E40001C3D11F41AE937C0113F69F51BE933C085
:102E5000143E11F411EE2FC0163F11F41FEE2BC0DB
:102E60001C3F11F415EF27C0113F11F41EEE23C0D3
:102E7000143C39F484E068E372E00E94E81614E040
:102E80001AC0163D39F485E060E472E00E94E8164D
:102E900015E011C01C3D39F486E068E472E00E9440
:102EA000E81616E008C01F3D31F487E060E572E0E7
:102EB0000E94E81617E0812F0E94C41503C0862FD8
:102EC0000E940A2F1F9108951F93CF93DF93182F0D
:102ED000EB0104C02196812F0E94FC1668816623B5
:102EE000C9F7DF91CF911F9108950F931F93DF933F
:102EF000CF93CDB7DEB7C055D0400FB6F894DEBF44
:102F00000FBECDBF9E01265A3F4F8E010F5F1F4F50
:102F1000C8016A966EAD7FAD6A97A9010E944F4CB9
:102F200068968FAD6897B8010E946417C05BDF4F49
:102F30000FB6F894DEBF0FBECDBFCF91DF911F91CA
:102F40000F9108950F931F93DF93CF93CDB7DEB703
:102F5000C055D0400FB6F894DEBF0FBECDBF9E0166
:102F6000265A3F4F8E010F5F1F4FC8016A966EAD04
:102F70007FAD6A97A9010E94334C68968FAD689720
:102F8000B8010E946417C05BDF4F0FB6F894DEBF34
:102F90000FBECDBFCF91DF911F910F9108951F9369
:102FA000CF93DF93182FEB0104C0812F0E94FC16F2
:102FB0002196FE0164916623C1F7DF91CF911F91A5
:102FC0000895E82FF0E0EF70F070E65CFC4FE491BC
:102FD0008E2F90E0089590E083709070009731F00C
:102FE000039711F48CE1089584E008958FE008952B
:102FF0008FE292E0089580914B0282FF05C080919C
:10300000310290913202089580912F029091300206
:10301000089590914B0291FD19C092FF05C08091D7
:103020002904823099F404C0809129048F3071F40E
:10303000109229049260977F90934B0210924F0256
:1030400080E090E060E070E00E944C1508958823D5
:10305000E9F082E068EA71E00E94E81683E060EB44
:1030600071E00E94E81684E068EB71E00E94E816C7
:1030700085E060EC71E00E94E81686E068EC71E0A3
:103080000E94E81687E060ED71E01CC082E068E60F
:1030900071E00E94E81683E068E771E00E94E8169C
:1030A00084E068E871E00E94E81685E060E971E07C
:1030B0000E94E81686E068E971E00E94E81687E061
:1030C00060EA71E00E94E816089580912E02833034
:1030D00014F010922E0280912E028F5F80932E02A8
:1030E0008150813041F0823061F0882379F481E0B1
:1030F00060E772E003C081E068E672E00E94E816D3
:10310000089581E060E672E00E94E8160895882341
:1031100021F082E060EF71E003C082E068EE71E0D0
:103120000E94E8160895882321F081E060EE71E0A6
:1031300003C081E068ED71E00E94E8160895FF92F7
:103140000F931F93DF93CF9300D000D000D0CDB763
:10315000DEB78C01F62EFE01319686E0DF011D926E
:103160008A95E9F7D8016D917C91CF010E94942650
:10317000F801808D918DA28DB38D282F2F772B8311
:1031800037E0B595A795979587953A95D1F7282F6C
:103190002F772C8327E0B595A795979587952A9546
:1031A000D1F781708D83FF2011F080688D8380E0DE
:1031B0006BE1AE014F5F5F4F0E94F42626960FB67B
:1031C000F894DEBF0FBECDBFCF91DF911F910F915D
:1031D000FF90089580935F020E94770E08952091DA
:1031E0004B0221FD0EC02B7F216020934B02909358
:1031F00032028093310270933A02609339020E9446
:10320000770E0895E0912F02F09130028E179F07FC
:1032100011F0EF2BF1F49B0140E050E0A9013327BE
:1032200022278091350290913602A0913702B09109
:103230003802A070B070282B392B4A2B5B2B2093BF
:1032400035023093360240933702509338020E9481
:10325000770E0895FC0180912F0290913002E817BB
:10326000F90711F510924E0260934D0260E070E094
:103270008091350290913602A0913702B0913802C8
:1032800080709070482B592B6A2B7B2B222311F0D6
:10329000616001C06E7F40933502509336026093A7
:1032A0003702709338020FC0809131029091320240
:1032B000E817F90751F410924E0260934D025093B3
:1032C0003A02409339020E94770E08951F93182FF7
:1032D00080E06CE00E940716112309F100D000D0B5
:1032E0000F92EDB7FEB7319682E0ADB7BEB711963B
:1032F0008C938DED92E09283818380914F0290E0D8
:103300008F779070948383830E9475170F900F902E
:103310000F900F900F9080E00E94C41505C082E0CE
:1033200068ED72E00E94CF171F910895EF92FF920F
:103330000F931F93182F80FF02C083E001C085EA1E
:103340000E94C415E12E11FF02C084E001C085EA8D
:103350000E94C415E2FE02C085E001C085EA0E9419
:10336000C415E3FE02C086E001C085EA0E94C415D0
:10337000E4FE02C087E001C085EA0E94C4151F91E7
:103380000F91FF90EF90089560913B0270913C0285
:1033900080913D0290913E02611571058105910574
:1033A00061F00E94E311882341F010923B021092D9
:1033B0003C0210923D0210923E0260913F027091D9
:1033C0004002809141029091420261157105810590
:1033D000910571F00E94E311882351F010923F0291
:1033E0001092400210924102109242020E94770E07
:1033F000609143027091440280914502909146028F
:10340000611571058105910561F00E94E311882322
:1034100041F0109243021092440210924502109221
:10342000460280914E0218166CF420914D0230E055
:103430002F7730708091500290E02817390714F0F0
:1034400010924E0280914E0287FF09C080914D027A
:1034500090E08F779070892B11F410924E0280913A
:103460004E0220912A0230912B0240912C02509161
:103470002D02882381F4211531054105510511F0F4
:103480000E94770E10922A0210922B0210922C02A8
:1034900010922D020895211531054105510539F08D
:1034A000CA01B9010E94E311882309F46CC080911C
:1034B0004E02181644F40E94740E833049F4809131
:1034C0004D028F5F03C080914D02815080934D0269
:1034D00080914E02813059F08F3F49F0823061F087
:1034E0008E3F51F028E833E140E050E009C020E38E
:1034F00035E740E050E004C020EE3EE240E050E01E
:10350000809150028E3781F48091F7039091F803F7
:10351000A091F903B091FA03F7E0569547953795D6
:103520002795FA95D1F721C08E3081F48091F70369
:103530009091F803A091F903B091FA03E4E0569555
:10354000479537952795EA95D1F70FC08091F703F6
:103550009091F803A091F903B091FA0375E05695A4
:103560004795379527957A95D1F7280F391F4A1F28
:103570005B1F20932A0230932B0240932C0250931E
:103580002D020E94770E089580914B0280FD25C088
:1035900060913B0270913C0280913D0290913E020D
:1035A000611571058105910521F00E94E3118823C1
:1035B000A1F0109232021092310210925202109237
:1035C00051021092300210922F0210924B02109270
:1035D00053020E94770E81E0089580E008951F93C2
:1035E000FC01009769F410924B0210923B0210927A
:1035F0003C0210923D0210923E020E94C41A48C042
:1036000070914B0271FD44C060934D02CA01A0E06D
:10361000B0E020913502309136024091370250914E
:10362000380220703070822B932BA42BB52B809303
:10363000350290933602A0933702B09338028091FE
:10364000F7039091F803A091F903B091FA03885120
:103650009C4FAF4FBF4F816080933B0290933C02E1
:10366000A0933D02B0933E0272FF09C071607B7F60
:1036700070934B02F0933202E093310207C07E7FD9
:1036800070934B02F0933002E0932F020E94770E6A
:103690001F910895DF92EF92FF920F931F93109165
:1036A0005F02112399F081E060E00E940716812FEC
:1036B00081500E94EA24BC0182E00E94CF17109240
:1036C0005F0288EE93E00E948E1202C0882319F0F8
:1036D0000E94FB1504C080E060E00E940716809104
:1036E0002F0290913002892BF9F00E943725FC01BE
:1036F00040912F0250913002828193818417950767
:1037000049F4218532858091510290915202281707
:10371000390751F0538342838091510290915202B4
:10372000928781870E941A2620912F0230913002C1
:1037300021153105C9F4109235021092360210920B
:1037400037021092380210924E0210923A021092F2
:10375000390210924D0210924F0280914B028F7EDF
:1037600080934B0210924C0280914B0282FD0DC05F
:103770008091470290914802A0914902B0914A027B
:103780000097A105B10531F430C082E067E373E032
:103790000E94CF178DB79EB707970FB6F8949EBFBC
:1037A0000FBE8DBFEDB7FEB7319682E0ADB7BEB7A5
:1037B00011968C9384E293E09283818380914702F7
:1037C00090914802A0914902B0914A028383948368
:1037D000A583B6830E947517EDB7FEB737960FB66F
:1037E000F894FEBF0FBEEDBF51C02115310531F475
:1037F00082E06DE173E00E94CF1721C000D000D0BD
:103800000F92EDB7FEB7319682E0ADB7BEB7119615
:103810008C9388E193E092838183348323830E9495
:10382000751780914B020F900F900F900F900F9093
:1038300080FF02C081E001C080E20E94C4151091A7
:103840004C020E94740E682F863008F0615063307D
:1038500091F480912F0290913002892B61F0612FB9
:1038600070E06370707003E0660F771F0A95E1F7F0
:1038700068587D4F08C070E013E0660F771F1A95F7
:10388000E1F768567D4F82E00E94CF1780E06CE040
:103890000E94071680914B0283FF12C000D000D017
:1038A0000F92EDB7FEB7319682E0ADB7BEB7119675
:1038B0008C9384E193E09283818380914F0211C0C5
:1038C00000D000D00F92EDB7FEB7319682E0ADB7D1
:1038D000BEB711968C9380E193E0928381838091AF
:1038E0004D0290E08F779070948383830E947517C8
:1038F0000F900F900F900F900F9080912F0290914A
:103900003002892B89F080914C028370813081F4E0
:1039100087E10E943714882339F080E00E94C415A3
:1039200080E068E272E05BC080E20E94C41559C08A
:1039300080E00E94C4150E943725FC01808185FF2C
:1039400043C080914D0287FF04C080E06CE271E0CB
:1039500003C080E060E371E040E024E00E94B11623
:1039600080914E028823E1F018163CF08E3F81F0E2
:103970008F3F94F48D3FA9F507C08230C9F08230A3
:103980009CF0833071F518C080E06CE471E017C0E2
:1039900080E068E471E013C080E064E471E00FC08F
:1039A00080E064E371E00BC080E068E371E007C091
:1039B00080E06CE371E003C080E060E471E044E02B
:1039C00024E00E94B1160DC080914D0287FF04C013
:1039D00080E06CE171E003C080E064E271E00E948D
:1039E000E8160E94740E813049F489E00E94072590
:1039F000AC0181E060E00E94611603C280914B023D
:103A000083FD06C080E060E040E050E00E941016B8
:103A100080914B0287FD03C000E010E014C080914C
:103A2000310290913202892B19F001E010E00BC0B5
:103A300080914C020E94EB1720E030E0853010F0BE
:103A400021E030E08901F02E81E060E00E9407165D
:103A50008091470290914802A0914902B0914A0298
:103A60000097A105B10509F429C18DE00E94371422
:103A7000882329F48EE00E943714882381F100D036
:103A80000F9282E0EDB7FEB7818384E093E09383E9
:103A900082830E9475170F900F900F908DE00E9407
:103AA0003714882369F081E060EE71E00E94E81627
:103AB00082E068EE71E00E94E81683E998E10CC0AC
:103AC00081E068ED71E00E94E81682E060EF71E04D
:103AD0000E94E81687E898E16CE271E0ECC087E0AC
:103AE0000E940725BC0182E00E94CF1787E00E9458
:103AF00007250E94134C182F04C080E20E94C415B1
:103B00001F5F1031D0F310914C02812F0E94EB17F0
:103B100090E0A0E0B0E0209147023091480240914F
:103B2000490250914A0282179307A407B5070CF483
:103B30004DC081E06BE00E940716609147027091D2
:103B4000480281E090E0A0E0B0E0062E04C0880FBB
:103B5000991FAA1FBB1F0A94D2F7209135023091FA
:103B60003602409137025091380282239323A423D6
:103B7000B5230097A105B10519F425EA30E002C08C
:103B800023E030E08DB79EB707970FB6F8949EBF3D
:103B90000FBE8DBFEDB7FEB7319682E0ADB7BEB7B1
:103BA00011968C938BEF92E092838183CB01638398
:103BB0009483368325830E947517EDB7FEB7379639
:103BC0000FB6F894FEBF0FBEEDBFC0C01370133028
:103BD00009F0BCC08FE00E943714882351F480E1C3
:103BE0000E943714882329F48CE00E94371488231C
:103BF00069F180E10E943714882321F081E060E6BA
:103C000072E003C081E068E572E00E94E81681E09E
:103C10006FE00E94071600D000D00F92EDB7FEB7FC
:103C2000319682E0ADB7BEB711968C9388EF92E0E3
:103C30009283818381E090E0948383830E9475174F
:103C40000F900F900F900F900F90DBC081E060E617
:103C500072E00E94E81681E06BE00E940716EDB763
:103C6000FEB739970FB6F894FEBF0FBEEDBF319681
:103C700082E0ADB7BEB711968C938FEE92E092833F
:103C8000818386E090E09483838387E090E096834D
:103C9000858381E090E0908787830E947517EDB758
:103CA000FEB739960FB6F894FEBF0FBEEDBF85E69E
:103CB00098E168EC70E00E944C15A3C0209131029D
:103CC000309132022115310539F100D000D00F9228
:103CD000EDB7FEB7319682E0ADB7BEB711968C93C3
:103CE0008AEE92E092838183348323830E94751746
:103CF0000F900F900F900F900F90809139028F715D
:103D00000E949619002321F08CE30E94C4152DC057
:103D100080E20E94C4151CC000D000D00F92EDB705
:103D2000FEB7319682E0ADB7BEB711968C9381EEA7
:103D300092E09283818383E592E0948383830E945F
:103D400075170F900F900F900F900F90FF2069F450
:103D500080913F0290914002A0914102B0914202B5
:103D60000097A105B10509F444C0809131029091FA
:103D70003202892BF1F580914C020E94EB178530BD
:103D8000C0F181E060E00E94071686E40E94C4153D
:103D9000B2E0EB2EF12C012D112DDD24D394809176
:103DA000350290913602A0913702B09138028E21EF
:103DB0009F21A023B1230097A105B10549F0B9E0E7
:103DC000BD1518F08D2D805D04C08D2D885001C06B
:103DD00085EA0E94C415D394E0E1DE1629F0EE0CCA
:103DE000FF1C001F111FDBCF80E20E94C41581E081
:103DF00006C0809135028F710E94961980E00E9462
:103E000027181F910F91FF90EF90DF900895CF93A7
:103E1000DF93EB0180934C02E82FF0E0EF70F0703D
:103E2000E65CFC4FE491E09350026115710559F096
:103E3000CB0160E070E043E552E00E94392DD09361
:103E40005202C09351020E94770EDF91CF910895E4
:103E5000AC0180914B028C7F80934B0210925202F6
:103E600010925102662309F045C01092530220912E
:103E70002F02309130022115310521F030933402A8
:103E800020933302109235021092360210923702BC
:103E90001092380210923A021092390210923202B5
:103EA000109231021092300210922F0210924E02A4
:103EB00010924C02109229044115510551F18FEFD7
:103EC000BA010E94EF2580914B0281FD22C0109221
:103ED0003502109236021092370210923802109278
:103EE0003202109231021092300210922F02109280
:103EF0004C020DC01092290460912F027091300283
:103F00008FEF0E94B62580914B0281FD02C090E0A8
:103F100001C091E080914B028B7F826080934B02C5
:103F2000892F0895EF92FF920F931F93DF93CF9302
:103F300000D000D000D0CDB7DEB77C01FE013196B5
:103F400086E0DF011D928A95E9F7F701208D318D1A
:103F5000428D538D2030F8E23F07F0E04F07F0E04C
:103F60005F072CF0D7015C968C9186FF7DC02030D6
:103F7000B0E43B07B0E04B07B0E05B070CF074C067
:103F8000F70162817381211531054105510509F45D
:103F90005DC06115710559F180819181A0E0B0E0AB
:103FA00082179307A407B50741F0CB01A0E0B0E06A
:103FB00082179307A407B507D1F4D7015C968C91BB
:103FC0005C978E7F5C968C935C976D917C918E0153
:103FD0000F5F1F4FC8010E94942680E065E0A80192
:103FE0000E94F426F7011382128211821082D701F7
:103FF0008D919C91A0E0B0E0F701208D318D428D34
:10400000538D82179307A407B50769F4848D91E057
:1040100089278B7F848FD70158961D921D921D9200
:104020001C925B9721C081E060E00E94071680E04F
:104030000E940725BC0182E00E94CF17F701648D22
:104040006470808D918D0E94281F09C0672B39F400
:10405000D7015C968C915C9784605C968C93F70199
:10406000108E118E128E138E26960FB6F894DEBF28
:104070000FBECDBFCF91DF911F910F91FF90EF90B9
:104080000895AF92BF92DF92EF92FF920F931F932A
:10409000DF93CF93CDB7DEB72C970FB6F894DEBF82
:1040A0000FBECDBF9C015E010894A11CB11C86E02F
:1040B000D5011D928A95E9F72531310509F49AC396
:1040C000263131052CF52C30310509F47DC12D3018
:1040D0003105ACF42A3031054CF4213031050CF0B7
:1040E000E3C32115310509F493C328C42A303105EF
:1040F00009F40CC42B30310509F020C4FEC3213172
:1041000031050CF0A2C22F3031050CF00DC333C2C3
:104110002A38310509F4F6C32B383105A4F42B31C4
:10412000310564F4293131051CF52631310509F4D6
:104130001BC32731310509F001C40BC123323105FE
:1041400009F0FCC3F2C32F3831054CF42D3831058A
:104150000CF011C22C38310509F0F0C3E9C1213946
:1041600031050CF4FBC22739310509F0E7C3E4C37C
:1041700080914B0283FF03C010914F0202C0109147
:104180004D0200E02931310509F401E0E0905002D0
:104190000E943725FC01F7800E943725FC018081B1
:1041A00084FF35C017FD05C080E0002309F481E0DD
:1041B000082F002311F001E02CC0812F90E08F77B1
:1041C0009070892B79F48091430290914402A091E0
:1041D0004502B09146020097A105B10519F4212FBF
:1041E0002058ADC08091F7039091F803A091F90396
:1041F000B091FA03845D9E4FAF4FBF4F809343024F
:1042000090934402A0934502B093460224C0002339
:1042100011F10E943725FC01808185FF07C0809144
:104220004E0283300CF08AC08F5F21C00E94740E52
:10423000833009F083C0812F90E08F7790702E2D0E
:1042400030E0821793070CF079C0FEE7EF16E1F536
:10425000FF20E1F439C00E943725FC01808185FFF1
:1042600009C080914E028E3F0CF468C0815080934B
:104270004E0264C0812F90E08F779070892B09F4F3
:104280005DC04EE7E41641F5FF2031F181E0F816FC
:1042900019F460E820E00EC0A2E0FA1619F46EE30B
:1042A00024E108C0B3E0FB1619F466E12AE002C07D
:1042B00060E820E8812F90E030E0002341F08F7724
:1042C0009070821793075CF4212F2F5F38C08F778F
:1042D0009070281739071CF0212F215030C0462F2D
:1042E00050E0812F90E08F779070481759071CF0AD
:1042F000212F2E7F04C0212F261B2C7F260F211754
:1043000019F0002319F41BC0002361F0822F90E004
:104310008F7790708417950714F482E001C084E0D1
:10432000280F0DC0822F90E08F77907048175907A3
:1043300014F082E001C084E0281B01C0212F80918D
:104340004B0283FF03C020934F02207820934D023D
:10435000F3C290914B0297FF21C088E08927809398
:104360004B0283FF0EC080914D0280934F028078F4
:1043700080934D0210924E0286E699E160E971E069
:104380000AC080914F0280934D0210924F0280E04C
:1043900090E060E070E00E944C15CEC280914C022B
:1043A0008370813029F480E068E272E00E94E816B0
:1043B00080914D028058807880934D0210924E0279
:1043C00080914B02877FAEC2809131029091320280
:1043D000009709F07DC0E0904702F09048020091FC
:1043E000490210914A021E141F04100611060CF017
:1043F0006FC0D0904C028D2D0E94EB1790E0A0E092
:10440000B0E08E159F05A007B1070CF458C081E0FD
:1044100090E0A0E0B0E00E2C04C0880F991FAA1F06
:10442000BB1F0A94D2F72091350230913602409199
:1044300037025091380282279327A427B52780930B
:10444000350290933602A0933702B09338028091E0
:104450004B02806880934B02E0E1EE16F104010507
:1044600011050CF4BAC160912F0270913002C501A0
:104470000E949426209135023091360240913702F5
:1044800050913802CA01AA27BB278F778B8377E127
:1044900056954795379527957A95D1F7822F8F773F
:1044A0008C8367E056954795379527956A95D1F7A0
:1044B0002D8380E06DE0A5010E94F4268EC1F3E01B
:1044C000DF22DF1609F038C28FE292E061E040C1DE
:1044D00060914B0267FF10C0892B71F08091390207
:1044E00090913A0221E030E08227932790933A029C
:1044F00080933902606119C0809135029091360233
:10450000A0913702B091380221E030E040E050E065
:1045100082279327A427B5278093350290933602EC
:10452000A0933702B09338026F7E60934B0204C2AF
:104530008091310290913202892B29F480914B02B3
:104540008F7780934B0280914B0285FFF5C180915C
:10455000470290914802A0914902B0914A02181670
:1045600019061A061B060CF0F9C08FE292E060E013
:104570000E949F18F3C086E0FE013796DF011D926E
:104580008A95E9F78091470290914802A0914902EB
:10459000B0914A020097A105B10509F454C0893FC2
:1045A000E7E09E07E0E0AE07E0E0BE070CF0C4C124
:1045B0008C0101501040000F111FC9018F779070BE
:1045C0000E9709F4016027FF23C01A8680914B02E1
:1045D00083FD05C080E090E060E070E004C086E606
:1045E00099E160E971E00E944C1581E060E671E0BC
:1045F0000E94E81682E068E671E00E94E8161092D8
:104600004702109248021092490210924A0202C0D8
:1046100081E08A87802F8F778F83C801880F892F49
:10462000881F990B91958F778887812F8295869522
:1046300086958370898780E066E0AE01495F5F4FB1
:104640000E94F42679C127FD77C1022F0D501091E9
:104650004B0217FF0AC08091310290913202892BE0
:1046600021F4213131050CF40C5F80914C020E9441
:10467000EB17081708F060C10430A0F08091F70331
:104680009091F803A091F903B091FA038C509E4FDA
:10469000AF4FBF4F80933F0290934002A0934102DF
:1046A000B093420217FF1DC08091310290913202F7
:1046B000892BB9F082E090E0A0E0B0E004C0880F60
:1046C000991FAA1FBB1F0A95D2F72091390230917A
:1046D0003A022827392730933A0220933902106191
:1046E00020C082E090E0A0E0B0E004C0880F991FF5
:1046F000AA1FBB1F0A95D2F72091350230913602CE
:10470000409137025091380282279327A427B5277A
:104710008093350290933602A0933702B09338020B
:104720001F7E10934B0208C180914702909148026E
:10473000A0914902B0914A020097A105B10509F480
:1047400084CF60E02F30310509F461E08FE292E020
:104750000E949F1880914B028062E4C080914B02BE
:104760008F7D80934B0239C080914702909148021F
:10477000A0914902B0914A020097A105B105B1F19B
:1047800080914B0282FD32C00E94740E833019F575
:1047900080915002282F30E040E050E080914702A5
:1047A00090914802A0914902B0914A022817390716
:1047B0004A075B0744F42093470230934802409332
:1047C000490250934A0280914D02807890914702AD
:1047D000892B80934D0210924E0210924702109244
:1047E00048021092490210924A02A6C080E060E29C
:1047F00043E00BC080914B0287FF04C080E060E281
:1048000042E003C080E060E240E00E940A2794C0DA
:1048100080914B0287FF12C0809133029091340245
:10482000009709F48BC0A0E0B0E08093470290931A
:104830004802A0934902B0934A021EC082FF21C0E1
:104840008091470290914802A0914902B0914A029A
:104850000097A105B105A9F486E00E946745809103
:10486000470290914802A0914902B0914A020097F4
:10487000A105B10509F462C08FE292E00E94921F87
:104880005DC08091470290914802A0914902B09189
:104890004A020097A105B10539F48FEF0E946745E0
:1048A00081E00E944A1B4AC079010027F7FC00956D
:1048B000102F6091470270914802809149029091B7
:1048C0004A022AE030E040E050E00E94D44BE60E7D
:1048D000F71E081F191FF0E0EF16F0E8FF06F0E0E2
:1048E0000F07F0E01F0754F5E0924702F0924802EC
:1048F0000093490210934A021FC08FE292E00E9487
:10490000921F1AC080914B028F770CC01092470201
:10491000109248021092490210924A0280914B0272
:104920008B7F806880934B0207C080914D02807816
:1049300080934D0210924E020E94770E2C960FB675
:10494000F894DEBF0FBECDBFCF91DF911F910F91C5
:10495000FF90EF90DF90BF90AF9008951F93182FB6
:10496000823118F02AEC37E032C00E943725FC0172
:104970002581243039F0253079F0812F90E02130E5
:10498000F1F414C0212F30E054E0220F331F5A9568
:10499000E1F7265B3C4F1BC0212F30E044E0220FA3
:1049A000331F4A95E1F726593B4F11C09C0194E013
:1049B000220F331F9A95E1F726573A4F08C09C0102
:1049C00084E0220F331F8A95E1F72655394FC9013C
:1049D0001F910895882319F02FE138E016C00E9436
:1049E0003725FC018581843029F0853031F0813014
:1049F00051F406C02BED37E008C02CEE37E005C0BF
:104A00002DEF37E002C02EE038E0C90108951F9372
:104A1000182F833218F02BE731E126C00E9437258A
:104A2000FC018581843029F0853051F08130B1F46A
:104A30000EC081E1189F90011124215D374F14C0F1
:104A400081E1189F900111242E57354F0DC081E14F
:104A5000189F900111242B52334F06C081E1189FFB
:104A600090011124285D304FC9011F91089581E6FE
:104A700092E0089590916102982309F091E0892FC6
:104A80000895ECEFFFEF25913591459154915070C9
:104A9000B901CA010895EFEFFFEF8491823029F444
:104AA000079902C080E8089582E00895FC01848D92
:104AB00081FD02C020E006C020E080819181892B29
:104AC00009F021E0822F0895FC01848D81FD02C050
:104AD00020E006C020E082819381892B09F021E04B
:104AE000822F0895F89488E181BD8BE081BDFFCFCE
:104AF000BF92CF92DF92EF92FF920F931F93CF93CB
:104B0000DF93082F6B01EA014115510529F10E943D
:104B1000F8177C0110E086E0B82E80E0602FA60137
:104B20000E94F426B0922A0402C00E947B0EC701A4
:104B3000FE010995882321F480912A048823A9F78E
:104B40000E94A026811110E0C701FE01099588236B
:104B500019F41F5F1A3008F3DF91CF911F910F9165
:104B6000FF90EF90DF90CF90BF900895DF93CF93A9
:104B700000D000D000D0CDB7DEB76115710531F19E
:104B80004115510519F1FE01319686E0DF011D92B4
:104B90008A95E9F7862F8F778983660F672F661FBF
:104BA000770B7195862F8F778A83842F8F778B83EE
:104BB000440F452F441F550B5195842F8F778C83BD
:104BC00082E0BF0144E655E20E94782526960FB6A2
:104BD000F894DEBF0FBECDBFCF91DF910895DF9374
:104BE000CF9300D000D000D0CDB7DEB761157105EE
:104BF000C1F0FE01319686E0DF011D928A95E9F74A
:104C0000862F8F778983660F672F661F770B7195C5
:104C1000862F8F778A8381E0BF0146E555E20E94A7
:104C2000782526960FB6F894DEBF0FBECDBFCF9184
:104C3000DF910895CF93DF93C0E0D0E0CE010E94D2
:104C4000584EFE01EF59FD4F6081861719F0CE01D5
:104C50000E94604EA8952196C032D10579F7DF9168
:104C6000CF9108958095909161029823909361026D
:104C70000E941A26089590916102982B90936102E8
:104C80000E941A260895809366020E941A260895AB
:104C900090916602973008F091E080E1E1E6F2E061
:104CA000DF011D928A95E9F788E180936502909370
:104CB00066020E941A26089581E692E060E070E0A4
:104CC00040E250E00E94484E80916302909164025D
:104CD0008F5F9F4F11F40E944826809166028730B3
:104CE00010F010926602EAEFFFEF9491892F815045
:104CF0008E3F10F490936F000895FC0120E090E047
:104D000037E08191982780E097FF03C0990F9327A0
:104D100001C0990F8F5F8830B9F72F5F283089F76E
:104D200097FD9095892F0895FC01862F8F778083BA
:104D3000660F672F661F770B71956F7761830895F4
:104D400080918902882319F01092890281E00895E8
:104D50002091030130910401909304018093030199
:104D6000C9010895E0918102F0918202309709F023
:104D7000099508958091020108950F931F93DF9381
:104D8000CF93CDB7DEB729970FB6F894DEBF0FBE2D
:104D9000CDBFDA0180910201806889836A83FE01B8
:104DA00033969E01275F3F4F109721F08D918F77AB
:104DB000808301C010823196E217F307A9F78E01B4
:104DC0000F5F1F4FC8010E947D268987C8010E947E
:104DD000E21029960FB6F894DEBF0FBECDBFCF917B
:104DE000DF911F910F9108950F931F93CF93DF933E
:104DF000082F162FEA0102C00E947B0E802F612F20
:104E0000AE010E94BD268823B9F3DF91CF911F9197
:104E10000F910895DF93CF9300D000D000D0CDB78D
:104E2000DEB7FE01319696E0DF011D929A95E9F713
:104E30004983AF010E94F42626960FB6F894DEBF90
:104E40000FBECDBFCF91DF910895FF920F931F93B7
:104E5000CF93DF93082FEB014115510519F42FEF84
:104E60003FEF4FC0809103019091040150930401E2
:104E700040930301909382028093810210928502F5
:104E80008EEF9FEF90938402809383023093880289
:104E90002093870210E094E0F92E002361F080E077
:104EA000602FAE010E94F42606C00E947B0E809106
:104EB0008602882311F0F0922A04909185029923AA
:104EC00021F480912A04882381F780918902882324
:104ED00019F01092890210E0992319F41F5F18301D
:104EE000E0F280918102909182029093040180937C
:104EF000030110928202109281022091830230916C
:104F00008402C901DF91CF911F910F91FF90089505
:104F100020E030E00E9425270895DF92EF92FF9273
:104F20000F931F93DF93CF93CDB7DEB729970FB6BB
:104F3000F894DEBF0FBECDBF8E010F5F1F4F23ED74
:104F4000E22E28E2F22EDD24D3941CC0C8010E9478
:104F50007D2699858917B1F41BC0D092890212C0B1
:104F60008091030190910401892B21F4F0920401B6
:104F7000E0920301E0910301F0910401309711F0F8
:104F8000C8010995C8010E940C11892BF9F604C0CB
:104F90008A81863029F7E1CF29960FB6F894DEBFD3
:104FA0000FBECDBFCF91DF911F910F91FF90EF907A
:104FB000DF9008952F923F924F925F926F927F926F
:104FC0008F929F92AF92BF92CF92DF92EF92FF9219
:104FD0000F931F93DF93CF93CDB7DEB729970FB60B
:104FE000F894DEBF0FBECDBF0E9441259B01AC01EE
:104FF00010E8612E1FE3712E812C912C6222732206
:1050000084229522B7E09594879477946794BA9513
:10501000D1F7A12CA0ECBA2EAFE1CA2ED12CA2223E
:10502000B322C422D522FEE0D594C794B794A794A6
:10503000FA95D1F7E12CF12CE0EE0E2F112DE222A2
:10504000F3220423152375E115950795F794E7944A
:105050007A95D1F76FE7262E312C412C512C222244
:105060003322442255222DC0A8958A81843049F5E7
:10507000CE0101960E947D269985891711F541C0C0
:105080008D8190E0A0E0B0E0681679068A069B0664
:10509000C1F48C8190E0A0E0B0E0A816B906CA0681
:1050A000DB0679F48B8190E0A0E0B0E0E816F90629
:1050B0000A071B0731F489818F778093020181E011
:1050C00007C0CE0101960E940C11892B69F680E081
:1050D00029960FB6F894DEBF0FBECDBFCF91DF91FA
:1050E0001F910F91FF90EF90DF90CF90BF90AF9006
:1050F0009F908F907F906F905F904F903F902F90F8
:1051000008958E8190E0A0E0B0E0281639064A06A6
:105110005B06B9F6B5CF0F931F93DF93CF93CDB74F
:10512000DEB729970FB6F894DEBF0FBECDBF209132
:1051300002012068298323E02A83282F2F772B83DD
:10514000880F892F881F990B91958F778C83862FD5
:105150008F778D83852F869586958E8367FF02C016
:1051600080648E83CA0103E0969587950A95E1F7DE
:105170008F778F83842F8295807788878E010F5F4A
:105180001F4FC8010E947D268987C8010E94021115
:1051900029960FB6F894DEBF0FBECDBFCF91DF9139
:1051A0001F910F910895AF92BF92CF92DF92EF922D
:1051B000FF920F931F93DF93CF9300D000D000D0C6
:1051C000CDB7DEB76C010E94F8175C01D6011196CD
:1051D0006C91862F90E0FC013397E332F10508F0E3
:1051E00098C2EA5BFF4FEE0FFF1F0590F491E02D90
:1051F0000994F60182810E94480FD60117968C917E
:1052000084700E94003285C2F50100811181D601AF
:1052100013968C91139790E09695982F88279795E1
:10522000879512962C9130E0822B932B0817190743
:1052300009F06FC20E94C41AC8010E94912F69C26E
:10524000F6018381E82FF0E0F695FE2FEE27F79523
:10525000E795D60112968C91129790E0E82BF92BE6
:1052600015968C911597382F330F330F20E0169633
:105270008C911697482F50E04F77507013E0440FF1
:10528000551F1A95E1F717968C9190E080779070F2
:1052900074E0959587957A95E1F7482B592B422B29
:1052A000532B683041F4CF01BA010E94EF1880916E
:1052B000290482602FC08091290481608093290491
:1052C000D60117968C9180FD05C0809129048260DB
:1052D00080932904D60114966C91149715968C919D
:1052E00086FD6068CF010E94EF1A0E94091811C262
:1052F000F601668170E07695762F6627779567953B
:10530000858190E0682B792B84810E94071F809112
:105310002904846080932904E8CFD60114964C9127
:10532000149750E015966C91159770E07695762F4E
:1053300066277795679516962C911697922F9295DA
:10534000990F990F907C80E0682B792B13968C91A4
:10535000139790E09695982F8827979587951296A2
:105360002C9130E0642B752B822B932B0E94021919
:10537000809129048860CECFF601628113818581F6
:10538000E82FF0E0D60116964C91169717968C915F
:105390001797282F30E014960C91E6FD0068FE2F39
:1053A000EE27FF0FFF0F50E04F77507083E0440F60
:1053B000551F8A95E1F7C90180779070B4E0959503
:1053C0008795BA95E1F7482B592B812F90E0969558
:1053D000982F88279795879570E04E2B5F2BE3E0F9
:1053E00036952795EA95E1F72170862B972B602F4C
:1053F0000E942A198EC1F50122A133A12115310580
:1054000069F0822F8F778983220F232F221F330B7E
:105410003195822F8F778A8318E00EC0D5018C9149
:105420008F7789838D919C91880F892F881F990B85
:1054300091958F778A8310E0F501848D80FD10614E
:105440000E944125262F2F772B83A7E096958795DD
:1054500077956795AA95D1F7262F2F772C83F7E0BC
:105460009695879577956795FA95D1F7262F2F779B
:105470002D83E7E09695879577956795EA95D1F71F
:105480006770612B6E838FEF6BE0AE014F5F5F4FF4
:105490000E94F4263EC10E9441257B018C019B01A4
:1054A000AC012F77307040705070D60114968C91FB
:1054B00090E0A0E0B0E0281739074A075B0709F041
:1054C0005EC1A801970120783F734070507067E07B
:1054D00056954795379527956A95D1F7F6018581B9
:1054E00090E0A0E0B0E0281739074A075B0709F011
:1054F00046C1A80197012070307C4F7150709EE02A
:1055000056954795379527959A95D1F7868190E0DE
:10551000A0E0B0E0281739074A075B0709F02FC160
:10552000278180E090E0A0EEB0E0E822F9220A2393
:105530001B2385E116950795F794E7948A95D1F793
:10554000822F90E0A0E0B0E087709070A070B07003
:10555000E816F9060A071B0709F011C18381682FB5
:1055600070E07695762F662777956795828190E033
:10557000682B792B6115710509F401C126952695D3
:105580002695122F20FF0BC0A5014C5D5F4FCB016C
:1055900060E070E00E94392DBC01009721F08091FD
:1055A00002010E94EF25D5018D919C911197892BC5
:1055B00009F4E5C011FFE3C05C968C915C978160B3
:1055C0005C968C93DCC0F601838190E09695982FD1
:1055D000882797958795228130E0822B932B909393
:1055E0002C0480932B0495C0D60113968C911397AD
:1055F00090E09695982F88279795879512962C91ED
:10560000129730E0822B932B90932F0480932E04DB
:1056100014968C91149780933C0415968C91159751
:105620008093300416968C918093310480912D04E0
:10563000816012C022E030E0F601E20FF31F8081AA
:10564000F901E05DFB4F80832F5F3F4F273031052D
:1056500099F780912D04826080932D045AC0F60141
:10566000828180933704838180933804848180937E
:105670003904858180933A0480912D048460ECCFB5
:10568000D60115968C911597882309F442C013967C
:105690008C911397482F50E05695542F44275795D7
:1056A000479514962C911497922F9295990F990FD4
:1056B000907C80E0482B592B12968C9190E0482BDF
:1056C000592B40FD02C067E601C062E7CA0196950A
:1056D00087950E94CC2F1DC00E947225F601828101
:1056E0000E94EA1816C0D60112968C91882329F0E0
:1056F0000E943725FC01848101C080E00E9484154E
:1057000008C090E0D60112968C91811191E090939F
:105710008602F601208130E02F77307080910201FF
:1057200090E02817390749F480912A04882329F04A
:1057300080912A04815080932A04D5015C968C9133
:1057400081FD06C080E090E060E040E050E015C0E0
:1057500084FF09C0F50182819381009721F0428581
:105760005385668D0AC0D50116964D915C911797A9
:105770008D919C9111975E966C910E948B28269634
:105780000FB6F894DEBF0FBECDBFCF91DF911F9152
:105790000F91FF90EF90DF90CF90BF90AF90089562
:1057A0009093840280938302209187023091880233
:1057B0002115310549F06115710531F0411551058B
:1057C00019F0C9010E941C4C81E080938502089564
:1057D00060E070E040E050E00E94D02B0895DF933D
:1057E000CF9300D000D000D0CDB7DEB7FE01319608
:1057F00026E0DF011D922A95E9F7282F2F772983CC
:10580000880F892F881F990B91958F778A838FEF47
:1058100063E1AF010E94F42626960FB6F894DEBF2E
:105820000FBECDBFCF91DF910895DF92EF92FF922F
:105830000F931F93DF93CF9300D000D000D0CDB74C
:10584000DEB7E62EFE01319626E0DF011D922A9595
:10585000E9F7282F2F772983880F892F881F990B25
:1058600091958F778A838FEF9FEF90932C0480938D
:105870002B0410E0FE2E0F2F35E0D32E16C08FEF35
:105880006E2D4F2D502F0E94F426D0922A0402C074
:105890000E947B0E80912B0490912C0497FF04C0F2
:1058A00080912A048823A1F71F5F80912B04909197
:1058B0002C0497FF02C01A3011F720912B0430916D
:1058C0002C04C90126960FB6F894DEBF0FBECDBFDB
:1058D000CF91DF911F910F91FF90EF90DF9008958E
:1058E00062E10E94152C089561E10E94152C089533
:1058F0008F929F92AF92BF92CF92DF92EF92FF92E0
:105900000F931F93DF93CF9300D000D000D0CDB77B
:10591000DEB7FC0179016115710509F48AC0211512
:10592000310509F486C06E010894C11CD11C86E0C3
:10593000D6011D928A95E9F7CB01880F892F881F20
:10594000990B9195BFE79B2E982214E1AFE7AA2E01
:10595000A6227FE7B72EB42265E0862E8E2F8F77A2
:105960008983EE0FEF2FEE1FFF0BF1958E2F8F77B0
:105970008A83163171F0173128F4143171F0153122
:1059800031F505C0173139F0183109F50AC090E03A
:105990000CC080E008C080E005C0AB829C82BD8264
:1059A00016C083E08D5F982F9D5FF701E90FF11D11
:1059B00080818B83892F8F5FF701E80FF11D908124
:1059C0009C838F5FF701E80FF11D80818D8310921A
:1059D0002C0410922B0400E015C08FEF612FA6015C
:1059E0000E94F42680922A0402C00E947B0E8091BD
:1059F0002B0490912C04892B21F480912A04882374
:105A0000A1F70F5F80912B0490912C04892B11F446
:105A10000A3019F780912B0490912C04892B49F0BE
:105A2000E0912B04F0912C041F5F193109F096CFFF
:105A300002C0E0E0F0E0CF0126960FB6F894DEBF9A
:105A40000FBECDBFCF91DF911F910F91FF90EF90CF
:105A5000DF90CF90BF90AF909F908F900895FC0102
:105A6000A62F9A0180E090E0BF014A2F0E94782C77
:105A70000895AF92BF92CF92DF92EF92FF920F9371
:105A80001F93DF93CF9300D000D000D0CDB7DEB707
:105A90009C018B017A0101978F5F934008F06CC0E5
:105AA000FE01319686E0DF011D928A95E9F7822F8B
:105AB0008F778983220F232F221F330B3195822F5B
:105AC0008F778A8310922D04DD24BE2ECF2E8FE097
:105AD000A82E1EC08FEF60E14B2D5C2D0E94F42696
:105AE000A0922A0402C00E947B0E80912D04873070
:105AF00021F080912A048823B1F780912D0487300A
:105B000031F082B790E08C599F4F0E948E12D3944F
:105B100080912D04873019F0BAE0DB16D9F6809118
:105B20002D04873021F4809130048F3759F401150A
:105B3000110511F0F8011082E114F104E9F0D70128
:105B40001C921AC00115110521F080913C04F80146
:105B50008083E114F10459F0D701E0E3F4E08BE035
:105B600001900D928150E1F7D7011B961C92209174
:105B70002E0430912F0402C020E030E0C9012696A7
:105B80000FB6F894DEBF0FBECDBFCF91DF911F914E
:105B90000F91FF90EF90DF90CF90BF90AF9008955E
:105BA00010923E0490913E0490933D0490913D04E8
:105BB000909360049091600490935F04119A109800
:105BC000199A189892E09BB9883008F087E0E82F7E
:105BD000F0E0EE0FFF1FE857FE4EA591B49165303F
:105BE00010F465E003C0693008F068E04F7D65504F
:105BF000660F453411F4606203C04F3409F46063EA
:105C0000223008F068608B2F992787FD9A958F7056
:105C100080939000A9B96093950088EB8AB980E0E1
:105C200090E008951F920F920FB60F9211248F9358
:105C30009F93EF93FF9390915F0480916004981776
:105C400011F4559812C0E0916004F0E0E35CFB4F62
:105C500084A18CB9809160048F5F809360048091EF
:105C60006004803210F010926004FF91EF919F91D8
:105C70008F910F900FBE0F901F9018951F920F924B
:105C80000FB60F9211242F933F938F939F93EF930F
:105C9000FF9320913D0480913E0430E090E0019715
:105CA0002817390741F080913D048F3179F48091B4
:105CB0003E04882359F480913E048F5F80933E0414
:105CC00080913E04803210F010923E04E0913D0439
:105CD000F0E08CB1E35CFB4F828380913D048F5FE9
:105CE00080933D0480913D04803210F010923D0479
:105CF000FF91EF919F918F913F912F910F900FBE48
:105D00000F901F90189527E0813D9207C0F12FE07A
:105D1000813A920710F481E01EC023E28932920793
:105D200010F482E018C026E3813B920710F483E070
:105D300012C026E48135920710F484E00CC028E8F4
:105D4000893B920710F485E006C0895D964D10F0FE
:105D500087E001C086E0789420E030E05E9902C0E0
:105D600020E030E02F5F3F4FA89597E220313907C0
:105D7000A8F368E04EE421E00E94D02D089580E071
:105D8000EACF8330C9F0843028F4813061F082306A
:105D900080F40CC08530B1F0853088F08630A9F0F1
:105DA0008730C9F415C020E639E017C020EB34E095
:105DB00014C020EC32E111C020E835E20EC020E42E
:105DC00038E30BC020E03BE408C020E036E905C022
:105DD00020E031EE02C020E030E0C901089539B181
:105DE00020919000922F80E0232F30E0282B392B38
:105DF00048E851E160E0FA01859194918217930798
:105E000029F06F5F4E5F5F4F6830A9F7862F0E94C1
:105E1000C12E0895482FA89503C0559A7894A89547
:105E200020915F048091600430E090E00197281792
:105E3000390799F380915F048F3121F480916004D8
:105E4000882359F3E0915F04F0E0E35CFB4F44A347
:105E50009FB7F89480915F048F5F80935F04809177
:105E60005F04803210F010925F049FBF559A80E06B
:105E700090E0089590913D0480913E04981719F4A4
:105E80002FEF3FEF15C0E0913E04F0E0E35CFB4FE5
:105E90009281F89480913E048F5F80933E048091BC
:105EA0003E04803210F010923E04292F30E07894A6
:105EB000C9010895CF92DF92EF92FF920F931F9343
:105EC000CF93DF93E82E162F042FF52E6AEC0E9455
:105ED000FC168E2D612F0E94FC16802F9F2DEC0149
:105EE00085E0C82ED12CCC0EDD1E0FC01881812F6D
:105EF0008A5C843028F48E2D6BEC0E94FC161F7097
:105F00008E2D612F0E94FC162196CC15DD0571F7B0
:105F1000DF91CF911F910F91FF90EF90DF90CF9085
:105F20000895DF93CF9300D000D000D0CDB7DEB777
:105F3000FE01319626E0DF011D922A95E9F799834B
:105F40008A8380E063E0AF010E945A2F26960FB645
:105F5000F894DEBF0FBECDBFCF91DF910895DF93E0
:105F6000CF9300D000D000D0CDB7DEB7FE01319680
:105F700096E0DF011D929A95E9F7898380E062E05F
:105F8000AF010E945A2F26960FB6F894DEBF0FBEBF
:105F9000CDBFCF91DF910895DF93CF9300D000D094
:105FA00000D0CDB7DEB7FE01319626E0DF011D92AD
:105FB0002A95E9F799838A836F776B8380E066E09F
:105FC000AF010E945A2F26960FB6F894DEBF0FBE7F
:105FD000CDBFCF91DF910895EF92FF920F931F9362
:105FE000DF93CF93CDB7DEB762970FB6F894DEBFDD
:105FF0000FBECDBF162F882309F094C18091940263
:106000008823B1F060918A0270918B0280918C029A
:1060100090918D026C5E7F4F8F4F9F4F0E94E311D6
:10602000882331F0109294021092950210929602F9
:106030008091F7039091F803A091F903B091FA03CE
:1060400080938A0290938B02A0938C02B0938D026E
:106050001A3C41F4109294021092950281E08093D0
:10606000960260C180919602882309F45BC11B3CB3
:1060700021F481E08093950255C1809195028111B0
:10608000106C1092950280919402E82FF0E0E65790
:10609000FD4F14838F5F80939402863008F442C1D1
:1060A0000E94F8178C0190918E02933009F4B4C0CD
:1060B000943030F4913059F1923008F055C00AC054
:1060C000953009F4C5C0953008F4B4C0963009F095
:1060D0001FC1E8C080E06CEC0E94FC16D801169647
:1060E0008D919C9117979C012E7F3F773695279530
:1060F00080FD3068F801868D8F83388729870E945C
:10610000740E8A871C861B8680E060E027C080E0D2
:106110006CEC0E94FC16D80111968C9111978F831C
:106120005C915D964C915D97242F30E02370307028
:1061300094968C91992787FD9095282B392B232BAA
:1061400011F480E001C080E858878987842F0E947D
:10615000E1178A871C861B8680E061E0AE01495FFB
:106160005F4F0E945A2FD8C090918F0280E02091FB
:106170009002BC01620F711D9091920280E020910B
:106180009302820F911DAC01440F551F4E7F5F7724
:1061900097FD41606115710519F4F8016081718105
:1061A000F0E460307F0708F0B3C0D8018D919C9176
:1061B0006817790739F4CB016091910220E00E94C1
:1061C0002A196DC0862F8F778983660F672F661F08
:1061D000770B7195862F8F778A8390919102892F03
:1061E0008F778B83852F869586958C8397FF02C04A
:1061F00080648C83CA0133E0969587953A95E1F7E0
:106200008F778D83842F829580778E8380E063E003
:10621000AE014F5F5F4F41C090918F0280E02091AF
:106220009002820F911D60E00E94281F882309F4CC
:106230006FC035C040918F02442329F0842F8250D3
:10624000823008F065C080E060E20E940A2727C023
:1062500030918F0220E080919002280F311DFE01C5
:10626000319686E0DF011D928A95E9F7822F8F77BC
:106270008983C901880F892F881F990B91958F7782
:106280008A83832F82958695869583708B838091F0
:1062900091028C8380E066E0AF010E94F42680E0EA
:1062A0006CEC38C030918F0220E080919002280F72
:1062B000311D8E01035F1F4FF80111929A95E9F786
:1062C000F22EE32EC801B9010E94942689E1B8019B
:1062D0004FE951E30E9488278C018235910569F0CE
:1062E0008335910524F48734910591F406C08736EF
:1062F000910519F08237910559F480E06CEC0E9409
:10630000FC16602F6F778F2D9E2D0E94CC2F04C01E
:1063100080E06DEC0E94FC1610929402109295029F
:106320001092960262960FB6F894DEBF0FBECDBFF4
:10633000CF91DF911F910F91FF90EF900895FC0195
:106340008181893121F0CF010E94B2260895848194
:1063500090E00E94E82B0895FB0157FD02C021E068
:1063600004C0509541955F4F20E08330910541F185
:106370008430910534F48130910501F1029751F593
:1063800023C08430910519F0059721F50AC0818159
:106390008F5F818390E084179507E4F0222351F00A
:1063A0000DC081818150818390E08417950794F01E
:1063B000222321F0842F815081830CC011820AC0D6
:1063C00012821382168A06C090E08281882309F423
:1063D00091E0928380E090E008958230910519F079
:1063E000039751F403C02FEF3FEF08C083E090E024
:1063F00040E050E00E94AC3120E030E0C901089557
:106400001F93182F0E94F817FC01848D112311F09F
:10641000806401C08F7B848F1F9108951F93CF9359
:10642000DF93EC018A81882309F470C081E060E089
:106430000E94071600D000D00F92EDB7FEB731963C
:1064400012E0ADB7BEB711961C9384E092E192833F
:1064500081838C819D81948383830E9475170F9023
:106460000F900F900F900F908B81843079F400D0B3
:106470000F92EDB7FEB7118380E092E193838283A0
:106480000E9475170F900F900F9018C000D000D089
:106490000F92EDB7FEB73196ADB7BEB711961C930C
:1064A0008CEF91E1928381838885838314820E949B
:1064B00075170F900F900F900F900F90898D9A8DF8
:1064C00097FD04C082E064EF71E10CC08E5F9F4FC6
:1064D00021F482E06CEE71E105C084E00E940725A2
:1064E000BC0182E00E94CF1781E0888F8E8B8B8168
:1064F000813058F0833020F08450823030F402C074
:1065000083E001C088E08F8B01C01E8ADF91CF91AC
:106510001F9108959C01FB018130910569F0823043
:1065200091051CF40097D9F027C083309105F1F054
:106530008530910509F517C08EEF9FEF928F818FFF
:106540004091A6025091A702CA0101978050944041
:1065500018F45583448310C0358324830DC0CB01C8
:106560000E940E3209C081E0838306C083E090E080
:1065700040E050E00E94AC3180E090E008951F932D
:10658000182F81E060E00E940716113049F01130A9
:1065900028F0123039F0133071F406C083E105C0E1
:1065A00084E103C085E101C086E10E940725BC01AA
:1065B00082E00E94CF171F9108951F93CF93DF931E
:1065C000EB018230910509F493C0833091051CF4EE
:1065D000892B31F0BBC0863091050CF0B7C075C077
:1065E00081E060E00E9407168A818823A1F000D034
:1065F00000D00F92EDB7FEB7319682E0ADB7BEB7CF
:1066000011968C9386EB91E1928381838C819D819D
:106610009483838346C020919702309198024091E1
:10662000990250919A02211531054105510509F44D
:1066300040C08DB79EB707970FB6F8949EBF0FBEA8
:106640008DBFEDB7FEB7319612E0ADB7BEB711966C
:106650001C938EEA91E19283818323833483458363
:1066600056830E9475176C817D818DB79EB7079602
:106670000FB6F8949EBF0FBE8DBF6115710509F46A
:1066800065C000D000D00F92EDB7FEB73196ADB720
:10669000BEB711961C9389EA91E19283818374833A
:1066A00063830E9475170F900F900F900F900F90BB
:1066B0004DC08C819D8197FF49C084E00E940725D1
:1066C000BC0182E00E94CF1741C08330910551F494
:1066D00010929702109298021092990210929A02C8
:1066E0001D821C82BE0142E050E00E94AC312EC0EF
:1066F0008A81882371F41D821C8283E08B838FEF53
:106700009FE39F838E8391E0988F85E08F8B9E8B94
:1067100017C01E8A8C819D810E942C4A609397022B
:10672000709398028093990290939A021B8261154C
:1067300071058105910521F48FEF9FEF9D838C8377
:1067400090E08A81882309F491E09A8380E090E0C8
:10675000DF91CF911F910895FF920F931F93CF93D5
:10676000DF93EC018B01F42E0E943725FC01C2302F
:10677000D10509F48BC0C330D10534F42097D1F092
:10678000219709F09BC00DC0C430D10509F463C046
:10679000C430D1050CF463C0C530D10509F08EC0FA
:1067A0005EC0FF2019F08485D8016DC08385F80193
:1067B000818384C081E060E00E940716FF2059F1C8
:1067C000D80111962C91EDB7FEB737970FB6F89414
:1067D000FEBF0FBEEDBF319682E0ADB7BEB71196DA
:1067E0008C9381EC91E192838183822F6AE00E94F5
:1067F000F34B83831482822F0E94F34B958316827E
:106800000E947517EDB7FEB737960FB6F894FEBF26
:106810000FBEEDBF53C000D000D00F92EDB7FEB752
:10682000319682E0ADB7BEB711968C938BEB91E1B8
:1068300092838183D80111968C9122E3829FC001BB
:106840001124948383830E9475170F900F900F90EB
:106850000F900F9033C0F80181818F3F79F1FF20B5
:1068600019F44BEE5FEF02C040E05FEFCE01B801DC
:106870000E94AC31FF2011F1D80111968C91119733
:106880008823E1F481E011968C9318C0D801129608
:106890008C911297882349F011968C91FF2011F06A
:1068A000848701C083870E941A2690E0F8018281C4
:1068B000882309F491E0D80112969C9380E090E03F
:1068C000DF91CF911F910F91FF90089541E00E94B9
:1068D000AC33089540E00E94AC3308951F93CF93EA
:1068E000DF93EB0182309105C1F18330910534F4DF
:1068F0000097C1F0019709F04CC005C086309105A2
:106900000CF047C025C00E943725FC01808185FF1F
:1069100002C082E003C084FF03C081E0898339C0E4
:10692000198237C081E060E00E9407168981825F8A
:106930000E94072500D00F9222E0EDB7FEB7218319
:10694000938382830E9475170F900F900F9021C040
:1069500043E050E00E94AC311CC08A81882399F04A
:106960000E943725FC0110811F7C8981813011F440
:10697000106103C0823009F410620E943725FC01C7
:1069800010830E941A2690E08A81882309F491E0FE
:106990009A8380E090E0DF91CF911F910895CF938B
:1069A000DF93EB018230910581F1833091052CF466
:1069B000009781F00197C9F504C086309105ACF5C8
:1069C0001FC00E943725FC0187818983843068F1CC
:1069D00019822BC081E060E00E9407168981865FE2
:1069E0000E94072500D00F9222E0EDB7FEB7218369
:1069F000938382830E9475170F900F900F9015C09C
:106A000044E050E00E94AC3110C08A81882339F004
:106A10000E9437252981FC0127830E941A2690E0D5
:106A20008A81882309F491E09A8380E090E0DF91E5
:106A3000CF9108951F93CF93DF939C01EB01823098
:106A4000910509F484C0833091053CF4009749F125
:106A50008130910509F0AEC005C0863091050CF07B
:106A6000A9C070C08C819D8101978C5F934010F00C
:106A70003D832C838CEF93E09F838E8311E01B83F7
:106A80001E8B83E08F8B188F8C819D810197880FDF
:106A9000991F0E941D481982039709F08BC0198322
:106AA00089C081E060E00E9407168B81813079F512
:106AB0002C813D818DB79EB707970FB6F8949EBF86
:106AC0000FBE8DBFEDB7FEB7319682E0ADB7BEB752
:106AD00011968C9385E091E09283818334832383A4
:106AE0002D5F3F4F368325830E94A2178DB79EB737
:106AF00007960FB6F8949EBF0FBE8DBF89818C5F3D
:106B00000E94AE24BC0182E00E94CF1753C000D087
:106B100000D00F92EDB7FEB7319682E0ADB7BEB7A9
:106B200011968C938FE091E0928381838C819D817B
:106B3000948383830E94A2170F900F900F900F9061
:106B40000F9038C042E050E00E94AC3133C08A81DF
:106B5000882399F02C813D818981882319F461E093
:106B600070E002C063E070E021503040C901880F3E
:106B7000991F0E94F2471A821DC08B81813019F43F
:106B80008A831E8A17C08C819D8101978C7F019614
:106B90009D838C830197880F991F0E941D4819823D
:106BA000039711F481E0898391E09B839E8B83E0BE
:106BB0008F8B988F80E090E0DF91CF911F910895A7
:106BC000CF93DF93EB018230910541F18330910542
:106BD0002CF4009789F00197E9F504C086309105FF
:106BE000CCF517C080E090E00E941D481982039701
:106BF00089F581E089832EC081E060E00E9407165C
:106C000089818E5F0E94AE24BC0182E00E94CF1772
:106C100021C042E050E00E94AC311CC08A81882330
:106C200099F081E060E00E94071682E069EC71E172
:106C30000E94CF178981882319F481E090E002C077
:106C400083E090E00E94CE4790E08A81882309F497
:106C500091E09A8380E090E0DF91CF910895CF9307
:106C6000DF93EB018230910509F450C08330910528
:106C700034F4009769F0019709F054C005C08630DC
:106C800091050CF04FC03DC00E941B4989834AC04A
:106C900081E060E00E94071669816623A9F48CE117
:106CA0000E94072500D00F9222E0ADB7BEB7119623
:106CB0002C93119713969C938E9312970E9475179D
:106CC0000F900F900F902EC000D000D00F92EDB714
:106CD000FEB7319682E0ADB7BEB711968C9388EDC2
:106CE00091E19283818385E0689FC00111249483A0
:106CF00083830E9475170F900F900F900F900F9045
:106D000011C049EC50E00E94AC310CC08A8188234C
:106D100019F089810E94F34890E08A81882309F460
:106D200091E09A8380E090E0DF91CF9108951F93E6
:106D3000CF93DF93EB01122F8230910519F183304D
:106D400091052CF4009761F0019779F504C0863025
:106D500091055CF512C0842F0E94044B898325C0E5
:106D600081E060E00E9407168981810F0E94AE24B5
:106D7000BC0182E00E94CF1718C042E050E00E94A0
:106D8000AC3113C08A81882351F08981882321F096
:106D9000842F0E94644B03C0842F0E94384B90E0E4
:106DA0008A81882309F491E09A8380E090E0DF9162
:106DB000CF911F91089544E026E00E9497360895F0
:106DC00041E020E00E949736089548E022E00E94CA
:106DD00097360895CF93DF93EB018130910569F0E9
:106DE000823091051CF4892B69F04CC082309105EA
:106DF00079F1039709F046C024C00E94D2489D83D0
:106E00008C8340C081E060E00E94071600D000D073
:106E10000F92EDB7FEB7319682E0ADB7BEB71196CF
:106E20008C938EED91E1928381838C819D819483FB
:106E300083830E9475170F900F900F900F900F9003
:106E400021C083E090E040E050E00E94AC311AC0E5
:106E50008A81882361F483E08B8384E390E09F83BD
:106E60008E8391E0988F82E08F8B9E8B05C01E8A67
:106E70008C819D810E94B14890E08A81882309F429
:106E800091E09A8380E090E0DF91CF910895CF93D5
:106E9000DF93EB018230910581F18330910534F469
:106EA0000097C9F0019709F044C005C086309105EC
:106EB0000CF03FC01DC00E942D46813051F0813042
:106EC00018F0833029F402C0198233C082E001C077
:106ED00083E089832EC081E060E00E9407168981EB
:106EE000885F0E94AE24BC0182E00E94CF1721C0BF
:106EF00044E050E00E94AC311CC08A81882399F0A4
:106F00008981813049F0813028F0823039F0833036
:106F100051F406C080E005C081E003C083E001C0F9
:106F200087E00E94F34590E08A81882309F491E08C
:106F30009A8380E090E0DF91CF910895CF93DF9323
:106F4000EB018230910549F1833091051CF4892BC6
:106F500029F02EC0863091055CF51AC08A818823FD
:106F600039F180E061E00E94071681E20E94072566
:106F7000BC0182E00E94CF1781E060E00E9407160A
:106F800089E10E940725BC0182E00E94CF1710C052
:106F900040E050E00E94AC310BC08A81882311F0A0
:106FA0000E943B4990E08A81882309F491E09A830A
:106FB00080E090E0DF91CF9108950F931F93CF93DE
:106FC000DF93FC018B01EA0180819181892B21F003
:106FD000858D8370833081F081E060E00E94071628
:106FE00085E00E940725BC0182E00E94CF1780E067
:106FF0000330110541F526C00E94740E833011F153
:107000000E94740E8230F1F00630110559F480E0D0
:1070100060E243E00E940A2781E090E0BE010E9406
:107020008A320EC081E060E00E94071686E00E946E
:107030000725BC0182E00E94CF171A821B821E8A9C
:1070400080E001C081E0DF91CF911F910F91089501
:10705000EF92FF920F931F93CF93DF938C01EB017D
:107060000E94F8177C01B801AE010E94DD37882329
:1070700009F4B1C00230110509F491C003301105C3
:1070800044F40115110549F10130110509F0A3C0BF
:107090000DC00430110509F45EC0043011050CF474
:1070A00076C00530110509F096C062C08EEF9FEFE3
:1070B0009A8F898F2091A6023091A702C90101976A
:1070C0008050944018F43D832C8302C01D830C83B0
:1070D00080E094E09F838E837EC08A81882309F4B8
:1070E0007AC081E060E00E9407162C813D8137FF65
:1070F00014C000D00F9282E0ADB7BEB711968C934A
:10710000119787EE91E113969C938E9312970E94AC
:1071100075170F900F900F9018C000D000D00F92ED
:10712000EDB7FEB7319682E0ADB7BEB711968C933E
:1071300083EE91E192838183348323830E947517C8
:107140000F900F900F900F900F9083E08F8B81E046
:10715000888F8E8B40C08C819D8101969D838C830E
:107160002E813F81821793077CF03D832C830CC0D6
:107170008C819D8101979D838C831816190624F0BC
:1071800081E090E09D838C8381E08B8324C083E049
:1071900090E0BE0140E050E00E94AC311CC091E0A4
:1071A0009B838A818823B1F02C813D8112161306BE
:1071B00094F421503040F7018081918160E041E0FA
:1071C00000E00E944B468C819D819093A7028093A2
:1071D000A60201C09A8380E090E0DF91CF911F91D9
:1071E0000F91FF90EF9008950F931F93CF93DF932C
:1071F000EC01062F142F8A818823F9F481E08B8318
:10720000643019F488E090E002C080E094E09F834D
:107210008E832C813D818E819F818217930724F478
:1072200081E090E09D838C8381E08A83083009F4BB
:10723000E0C080E00E94480FDCC08C819D8190936B
:10724000A7028093A602643009F1653060F46130D2
:1072500009F49EC06130D0F0623009F49BC0633005
:1072600009F0C7C0C4C0673009F492C0683038F470
:10727000653009F48DC0663009F0BBC007C06830C6
:1072800009F467C0693009F0B4C082C08B818150B5
:10729000823080F58EEF9FEF9A8F898FCE010E940A
:1072A0000E3281E06AE00E94071681E10E94072504
:1072B000BC0182E00E94CF17043051F0063069F023
:1072C000002391F48C819D8101970E9423470AC07D
:1072D0008C8181500E94504705C08C819D8101970F
:1072E0000E941E479A8F898F898D9A8D97FD56C06F
:1072F000888754C081E06AE00E94071682E10E94FC
:107300000725BC0182E00E94CF17043061F00630EF
:10731000B9F0002309F042C08C819D8101976885F6
:107320000E94EF4613C08C819D81893091051CF02D
:107330008FEF9FEF0BC0815068850E94284706C0E1
:107340008C819D81019768850E94E8469A8F898F7C
:1073500025C00E94F817FC0140815181411551055B
:10736000E9F0858D83708330C9F42C813D8121152E
:107370003105A1F08B818150823080F02150304066
:10738000CA01612F40E008850E944B461B8231C034
:1073900084E02EC08B818150823010F481E028C0BF
:1073A00081E06AE00E9407168B81863071F481E1EA
:1073B0000E940725BC0182E00E94CF178C819D812D
:1073C000019769850E94A3470EC082E10E940725AC
:1073D000BC0182E00E94CF178C819D810197698555
:1073E000498D0E9471479A8F898F86E001C087E09E
:1073F0008B83DF91CF911F910F9108950F931F936E
:10740000CF93DF93EC018B010E94F817BE01A80116
:107410000E94DD378823F1F0C230D10549F0C43035
:10742000D105A1F4C80169E040E00E94F43812C01F
:10743000C80168E040E00E94F438F80183818823A5
:1074400049F40E9403162FEF3FEF06C0CE01B801AA
:107450000E948A3220E030E0C901DF91CF911F9174
:107460000F9108958230910531F08430910549F4EF
:10747000CB0167E002C0CB0166E040E00E94F43837
:1074800002C00E948A3280E090E008958230910527
:1074900031F08430910549F4CB0165E002C0CB01A5
:1074A00064E040E00E94F43802C00E948A3280E02A
:1074B00090E008958230910531F08430910549F4CF
:1074C000CB0161E002C0CB0160E040E00E94F438F3
:1074D00002C00E948A3280E090E008951F93182F26
:1074E0001816B4F480E00E94BF3280E090E0612F73
:1074F0000E94EF46892B39F48CE190E065E040E092
:107500000E94714707C0812F0E949346892B11F07A
:1075100082E001C083E00E94BF3284EF91E00E94CC
:107520008E121F910895CF92DF92EF92FF920F93E8
:107530001F93CF93DF937B018130910571F08230EF
:1075400091051CF4892B89F0D0C08230910509F493
:1075500052C0039709F0C9C047C08FEF9FEFDB010E
:1075600015969C938E931497C0C0FB01828188234B
:1075700009F4BBC081E060E00E940716D7011496B1
:107580002D913C91159737FF10C000D00F9282E0EB
:10759000EDB7FEB781838EE092E1938382830E94F0
:1075A00075170F900F900F9018C000D000D00F9259
:1075B000EDB7FEB7319682E0ADB7BEB711968C93AA
:1075C0008AE092E192838183348323830E9475173A
:1075D0000F900F900F900F900F9085E0F701878B21
:1075E00081E0808F868B81C083E090E040E050E0B6
:1075F0000E94AC317AC0DB0112968C9112978823DD
:1076000099F11496CD91DC911597C038D10520F4ED
:107610008C2F0E946E3A2FC0B0E4C030DB0708F018
:107620006FC080E00E94BF326E016D2D606C80E102
:1076300090E00E94EF46892B09F062C081E190E062
:107640006C2F0E94EF46892B09F05AC08CE190E024
:1076500065E041E00E94714783E00E94BF3284EF01
:1076600091E00E948E1207C081E00E94BF3281E04B
:10767000D70112968C93F7018481958101978F37FA
:10768000910550F480E090E00E942347D7011596C1
:107690009C938E93149715C080E190E00E9423473D
:1076A000182F00E0F7011583048381E190E00E9428
:1076B0002347082B192B1F73D70115961C930E9384
:1076C0001497F70184819581805098423CF08FEFA8
:1076D0009FEFD70115969C938E93149781E0F70145
:1076E00083838FEF97E29783868380E090E0DF913A
:1076F000CF911F910F91FF90EF90DF90CF90089561
:1077000082E0ABCFCF93DF93EB018230910509F498
:107710004CC08330910509F441C0892B09F05DC04C
:107720008A81882309F459C081E060E00E9407162D
:107730002C813D8137FF14C000D00F9282E0ADB79D
:10774000BEB711968C93119789E192E113969C93A1
:107750008E9312970E9475170F900F900F9018C07C
:1077600000D000D00F92EDB7FEB7319682E0ADB7F2
:10777000BEB711968C9385E192E192838183348325
:1077800023830E9475170F900F900F900F900F900A
:1077900083E08F8B81E0888F8E8B1FC083E090E029
:1077A00040E050E00E94AC3118C08A81882321F06B
:1077B0008C810E946E3A05C081E00E94BF3281E058
:1077C0008A8380E090E00E9423479D838C8381E040
:1077D0008B838FE790E09F838E8380E090E0DF9142
:1077E000CF910895CF93DF93EB018230910509F497
:1077F0008FC08330910534F40097B1F0019709F000
:107800008CC00CC08430910509F46DC084309105A2
:107810000CF477C0059709F080C06BC081E090E060
:107820000E948A32198679C08A81882309F475C03A
:1078300081E060E00E9407168B81882331F482E0AA
:107840006DE272E10E94CF1725C08DB79EB70797F2
:107850000FB6F8949EBF0FBE8DBFEDB7FEB7319641
:1078600082E0ADB7BEB711968C938EE192E1928320
:1078700081838C819D81948383838985858316820E
:107880000E9475178DB79EB707960FB6F8949EBFE6
:107890000FBE8DBF898D9A8D97FD0AC082309105EC
:1078A0001CF0029729F402C0805D03C08FE301C081
:1078B00085E40E94C41581E0888F8E8B8B81863091
:1078C00059F0873020F48150823058F403C087305B
:1078D00041F404C086E003C08CE001C08EE08F8BD1
:1078E0001CC01E8A1AC08B81863041F4CB0163E034
:1078F00011C08B81863011F481E001C086E08B835A
:107900000CC083E090E040E050E00E94AC3105C044
:10791000CB0162E040E00E94F43880E090E0DF912B
:10792000CF910895AF92BF92CF92DF92EF92FF92E4
:107930000F931F93CF93DF938C01EB01823091055E
:1079400009F491C0833091053CF4009771F08130C7
:10795000910509F0A1C05DC08330910509F455C0BF
:10796000863091050CF098C06CC08A81882309F498
:1079700093C080919B02882309F48EC081E060E06F
:107980000E94071600D000D00F92EDB7FEB73196D7
:1079900082E0ADB7BEB711968C9382E093E19283FB
:1079A00081838C819D81948383830E9475170F90BE
:1079B0000F900F900F900F9089810E9490485C016A
:1079C000C12CE0E8DE2E70E8E72EF12C00E010E09C
:1079D000C6018A219B21892B11F424E001C026E0F5
:1079E000C7018A219B21892B09F02F5F822F0E94DA
:1079F000C415F694E7940F5F1F4F0830110519F076
:107A0000D694C794E5CF1E8A47C01E8A81E00E94A3
:107A100048480E94D24880939B0284E068E072E06C
:107A20000E94E81685E060E172E00E94E81686E0B8
:107A300068E172E00E94E81687E060E272E00E946E
:107A4000E81640919B02C801BE0150E00E94AC3193
:107A5000898190E001969D838C838B818230E1F453
:107A600088E08B8319C08A81882389F481E090E0C3
:107A70009D838C8380919B028E831F8211E01A83E9
:107A800080E00E944848188F85E08F8B1E8B88E02D
:107A90008B838C818150898380E090E0DF91CF914E
:107AA0001F910F91FF90EF90DF90CF90BF90AF901C
:107AB00008951F9380919D02803178F010929D026D
:107AC00010929C0281E061E00E94071610E085EAB6
:107AD0000E94C4151F5F1F30D1F781E060919D02A5
:107AE0000E94071680919C02813039F0813018F095
:107AF000823091F406C085E001C084E00E94C41584
:107B00000BC080E20E94C41585E00E94C4158091DC
:107B10009D028F5F80939D0280919C028F5F809376
:107B20009C02833010F010929C021F9108950F93D5
:107B30001F93CF93DF938C010E94FB17EC010097FA
:107B400031F482E061E472E10E94CF1718C000D0E6
:107B500000D00F92EDB7FEB7319682E0ADB7BEB759
:107B600011968C938DE392E192838183D483C383B6
:107B70000E9475170F900F900F900F900F900115A6
:107B8000110521F082E0B8010E94CF17CE01DF91EC
:107B9000CF911F910F9108950F931F93CF93DF9370
:107BA0008C010E94F817EC010115110521F002303B
:107BB0001105D9F518C080E090E00E94973D892B0F
:107BC000A1F181E060E00E9407168AA19BA1892BA8
:107BD00011F081E001C082E00E940725BC0182E033
:107BE0000E94CF1722C08A819B81892BF1F4888162
:107BF0009981892BD1F08AA19BA1892BB1F081E0D9
:107C000060E00E94071683E00E940725BC0182E025
:107C10000E94CF1784EF91E00E948E128AA19BA14F
:107C20000E94EF2B1BA21AA21CA280E090E0DF9121
:107C3000CF911F910F9108950F931F93CF93DF93CF
:107C4000EB018230910509F4A1C0833091053CF429
:107C5000009709F43EC0019709F0D4C00CC08430ED
:107C6000910509F444C0843091050CF488C005974F
:107C700009F0C8C061C00E94F817FC0180819181A1
:107C8000892B09F4BFC09F012C5D3F4FAE014B5EB5
:107C90005F4FDE011A9660E217C0F90180818823E8
:107CA00059F0E7E4F2E19491981721F03196992385
:107CB000D1F702C08C9301C06C93F90180818823B5
:107CC00011F02F5F3F4F1196A417B50730F31C92A8
:107CD00099C080E090E00E94973D81E060E00E94C2
:107CE00007162A9682E0BE010E9464178BC0898124
:107CF000A82FB0E0FB01EA0FFB1F228547E452E109
:107D0000FA0180E09491921731F03196992311F0A5
:107D10008F5FF8CF8FEF8F5FE82FFF27E7FDF0959C
:107D2000E95BFD4E8491882311F4FA018491AC0F34
:107D3000BD1F1A968C9366C08981A82FB0E0FB0105
:107D4000EA0FFB1F2285E7E4F2E180E094919217AD
:107D500029F03196992339F08F5FF8CF882319F0F5
:107D6000E82FE15001C0EFE2FF27E7FDF095E95B66
:107D7000FD4EE491AC0FBD1F1A96EC9343C083E017
:107D800090E04AE050E00E94AC313CC00E94F817FD
:107D90008C01FC0182819381892BA1F58A81882342
:107DA00049F489E08B8381E0888F19821F8A8A8356
:107DB0008E8B28C089818F5F89838F8B8B3010F1E8
:107DC0001B821A821E8A98012C5D3F4FD901FE0149
:107DD0003A968CE001900D928150E1F7F80182A172
:107DE00093A160817181009721F0458D0E94782CCC
:107DF00006C0CB01F801658DA9010E942F2DF80165
:107E000093A382A380E090E0DF91CF911F910F9127
:107E100008956F927F928F929F92AF92BF92DF925E
:107E2000EF92FF920F931F93CF93DF93EC017B01AF
:107E30000E94F8178C01C230D10509F47EC0C3300E
:107E4000D10534F4209719F1219709F0E5C005C058
:107E5000C630D1050CF0E0C031C0FC01258D922F59
:107E60009370848D86FF04C0992329F494E003C0A5
:107E7000992309F491E0269526952370235083E0F9
:107E8000989FC0011124280FF7012183C5C081E00C
:107E900060E00E9407168CED92E10E94973D892BCD
:107EA00009F4BAC0F70161818AE0689FB00111242A
:107EB00068587D4E82E00E94CF17AEC0FC01848DD1
:107EC00086FD03C049E050E002C04AE050E0CE0128
:107ED000B7010E94AC31F801808191818F3F9105FB
:107EE000B9F0B0F0F7018181882311F486E0818335
:107EF000F801848D86FD06C0F7018181863010F47B
:107F000088E08183F7018181863010F489E08183E4
:107F1000F801808191818050984208F47DC0F7017A
:107F20008181882311F489E08183F701818189307F
:107F300008F072C089E081836FC0FC018281938167
:107F4000892B09F069C0F7018281882309F45CC09C
:107F5000F801608071806114710409F45DC0858D41
:107F60000E94E117EC01F7014181842F63E00E9438
:107F7000F34B292F30E0220F331F220F331F842FA2
:107F80000E94F34BD82ED394D22AF4E0DF1609F4E2
:107F9000DD24F80182A093A08D2D0E94E117F80145
:107FA000268D422F50E04F775070BC01649FC00176
:107FB000659F900D749F900D1124BE010E94FF4B90
:107FC0002078262B268FE7012A96F4E2AF2EB12CDB
:107FD000A00EB11ECE01B5010E942C4CC3016D2D27
:107FE0000E94904B8114910459F0F80160817181D5
:107FF000C401458D9E010E94782CF80193A382A3B1
:10800000C501BE010E942C4C90E0F70182818823BB
:1080100009F491E0F701928380E090E0DF91CF9145
:108020001F910F91FF90EF90DF90BF90AF909F90C6
:108030008F907F906F900895AF92BF92CF92DF9212
:10804000EF92FF920F931F93DF93CF930F92CDB7D1
:10805000DEB77B018230910509F46CC08330910555
:1080600034F40097F1F0019709F0DFC00CC08430C0
:10807000910509F449C0843091050CF454C005976A
:1080800009F0D3C047C09B01265F3F4FC90160E2A2
:1080900070E04BE050E00E94254CD70155961C92B1
:1080A000C4C0FB018281882309F4BFC08181882379
:1080B00009F4BBC08B01065F1F4F90E060E070E0E9
:1080C000A8010E94392D00D000D00F92EDB7FEB765
:1080D000319622E0ADB7BEB711962C932FED32E169
:1080E00032832183948383830E9475170F900F90AE
:1080F0000F900F900F9081E060E00E94071682E0E1
:10810000B8010E94641791C0FB01818190E00E9438
:10811000742C05C0FB01818190E00E94702CD70176
:1081200011968C9382C083E090E040E050E00E9482
:10813000AC317BC090E0FB018281882309F491E09F
:10814000D70112969C930E94F8178C01F701828147
:10815000882371F0D80192968D919C919397009706
:1081600029F480E090E00E94742CF70181835DC0C7
:10817000BAE0AB2EB12CAE0CBF1CD70111968C917E
:1081800090E0BE016F5F7F4FA5010E94392D6C0109
:10819000F801848D82FF08C0C601A0E0B0E0808FA6
:1081A000918FA28FB38F3EC0D8018D919C91119772
:1081B000009721F015969C938E931497F8011386DF
:1081C000128613821282D80116961D921D921D925C
:1081D0001C92199711961C921E925C968C915C973A
:1081E0008C7F5C968C938FEFB6010E94EF25F8018F
:1081F00080819181892B21F0C60169810E94904B79
:10820000D8018D919C91892B69F0C8018496B501A4
:108210000E942C4CF7018181D80192968C93929701
:1082200093961C922FEF3FEF02C020E030E0C9018F
:108230000F90CF91DF911F910F91FF90EF90DF9002
:10824000CF90BF90AF9008950F931F93CF93DF937C
:10825000EC018B01009731F097FD40C00297029727
:10826000E8F536C081E060E00E940716D80112965A
:108270008C91882359F482E065EF72E10E94CF1758
:1082800082E06FEE72E10E94CF1722C00E9441256A
:10829000EDB7FEB737970FB6F894FEBF0FBEEDBF30
:1082A000319622E0ADB7BEB711962C9323EE32E1A2
:1082B0003283218363837483858396830E94751739
:1082C000EDB7FEB737960FB6F894FEBF0FBEEDBF01
:1082D000CE01B80140E050E00E94AC3180E090E077
:1082E000DF91CF911F910F910895CF93DF93EB0111
:1082F0008230910509F44AC08330910534F4009727
:1083000099F0019709F056C005C0863091050CF030
:1083100051C037C00E943725DC0114968C9163E070
:108320000E94F34B898346C081E060E00E940716FB
:10833000998183E0989F802D11240E94841582E00A
:1083400090E00E948E1281B763E00E94F34B898314
:1083500000D000D00F92EDB7FEB7319692E0ADB7E6
:10836000BEB711969C932EEF32E132832183838333
:1083700014820E9475170F900F900F900F900F901E
:1083800019C04FEE5FEF0E94AC3114C08A81882380
:1083900059F00E943725298143E0249F9001112440
:1083A000FC0124830E941A2690E08A81882309F424
:1083B00091E09A8380E090E0DF91CF910895CF9390
:1083C000DF93EB0182309105C9F1833091053CF4D4
:1083D000009751F08130910509F058C029C08630CE
:1083E00091050CF053C024C08A81882309F44EC043
:1083F00080E061E00E9407168981845F0E94AE24BC
:10840000BC0182E00E94CF1781E060E00E94071665
:108410006981623020F08AE10E94072504C0862F1E
:10842000805F0E94AE24BC0182E00E94CF172EC064
:10843000BE0142E050E00E94AC3128C08A8188230E
:1084400019F18981823018F48E5F89831FC081E021
:1084500060E00E9407168981833051F487E10E9411
:108460000725BC0182E00E94CF170E94D24509C0B7
:1084700088E10E940725BC0182E00E94CF170E947C
:10848000B2452FEF3FEF04C081E08A8320E030E067
:10849000C901DF91CF910895CF92DF92EF92FF92C1
:1084A0000F931F93CF93DF937C01162F0E94FB1530
:1084B0000E9437256C01173208F06AC0C12FD0E046
:1084C0008E01000F111F000F111F0C0F1D1F0D5EDD
:1084D0001E4FD70112968C91882311F080E001C0C5
:1084E00081E00E94C415F6018581843059F0853001
:1084F00089F0BE0124E0660F771F2A95E1F78130ED
:10850000B1F412C094E0CC0FDD1F9A95E1F7C45F7F
:10851000DC4E07C084E0CC0FDD1F8A95E1F7C4581C
:10852000DA4E82E0BE0106C06452784E02C0645C3E
:10853000754E82E00E94CF17D70112968C91882346
:1085400089F4F801848187FD0DC081E060E00E941C
:108550000716D80114968C910E940725BC0182E071
:108560000E94CF17D8011296ED91FC911397309786
:1085700021F080E090E0B7010995F7018689882312
:1085800029F0808D67890E94AB1602C00E940316F5
:10859000DF91CF911F910F91FF90EF90DF90CF90DF
:1085A00008952F923F924F925F926F927F928F9297
:1085B0009F92AF92BF92CF92DF92EF92FF920F9372
:1085C0001F93DF93CF93CDB7DEB76B970FB6F894B9
:1085D000DEBF0FBECDBFD82E45E2481708F45CC2FF
:1085E000DE0111968BE1FD0111928A95E9F7A895BC
:1085F0008D2D90E0FC01EE0FFF1FEE0FFF1FE80F27
:10860000F91FED5EFE4F0280F381E02D309721F0DF
:1086100081E090E0BD0109958E010F5F1F4FC801F9
:108620006D2D0E944C420E94F8174C0158018EEFAC
:10863000682E8FEF782E0FEF402E0FE7502E1BE0A5
:10864000212E312C2C0E3D1EF5E0DF9E80011124E1
:10865000B3E1EB2EB1E0FB2EE00EF11E0E947B0E8B
:108660000E945B149C018B30910509F4D1C08C30C1
:1086700091058CF48A3091050CF02DC18130910563
:108680000CF04BC14FEF8F3F940709F4F6C10097F0
:1086900009F433C1E3CF8731910509F4B9C08831BA
:1086A000910544F48531910509F4CAC186319105DB
:1086B000A9F6CFC18A31910509F450C082329105E3
:1086C00009F4E5C18931910549F68B81882369F068
:1086D000D7011296ED91FC911397309719F084E031
:1086E00090E0ABC18A818F5F48C01F8AF801ED5EC0
:1086F000FE4F1081A5E0EA2EF12CEE0EFF1ED39462
:108700000E94F817FC01848D86FD0AC0F2E0DF1696
:1087100039F485E090E0E80EF91EF3E0DF2E03C0A7
:1087200095E29D152CF0D7018C91811709F45EC05C
:10873000A3E1B1E060E0E12FFF27E7FDF0958C9128
:1087400090E08E179F0711F4D62E50C06F5F6632EF
:1087500011F01596F4CFDD24DA9448C08B8188237C
:1087600071F0D7011296ED91FC911397309719F0A3
:1087700085E090E062C18A8181508A8388C11F8A26
:108780000D5E1E4FF801C080EBEFEE2EEFEFFE2ED8
:10879000E00EF11EDA940E94F817DC015C968C91D1
:1087A00086FD0BC0B2E0DB1641F47801E6EFFFEF87
:1087B000EE0EFF1EDD24D39402C0D7FC04C0D70107
:1087C0008C918C1599F0ECECF1E075E2D72E2C2D04
:1087D000332727FD3095808190E08217930731F091
:1087E000DA94BFEFDB1611F03597F5CF8D2D90E0C1
:1087F000FC01EE0FFF1FEE0FFF1FE80FF91FED5EEC
:10880000FE4F0280F381E02D309709F05AC03FC13E
:10881000F70191819923E9F1A92FB0E0FD01E2561A
:10882000FD4F80811816BCF0E3E1F1E020E0492F14
:10883000552747FD5095808190E08417950711F4E6
:10884000822F06C02F5F263211F03596F4CF8FEFBE
:10885000A256BD4F8C93D7011196EC91F0E0E256F1
:10886000FD4F80810E94D142282F332727FD30956C
:10887000F7018181E82FF0E0E256FD4FC90137FF93
:1088800004C088279927821B930B808337FFFFC082
:108890000DC0D7011296ED91FC9113973097A1F07E
:1088A00082E090E0B501099597FF02C0D194F5C030
:1088B0008B81882309F0EBC0D7011296ED91FC91D2
:1088C000139781E090E0B9C090E08B81882309F490
:1088D00091E09B83DCC08B81882309F4DEC0D70143
:1088E0001296ED91FC911397309729F083E090E078
:1088F000B5010995DDCF1B82CAC08C81813009F496
:10890000A3CE883051F481E00E9448488A810E94B9
:10891000904880E00E944848BAC08C81853009F4B4
:1089200061C0863070F4823041F1833020F48130B0
:1089300009F0ADC012C0833081F0843009F0A7C0C7
:108940004EC0873009F463C0873008F45AC08830BD
:1089500021F0893009F09BC060C08F819885892BF8
:1089600011F458864F828F819885821793070CF4F3
:108970008EC01E821D8282E08C838D819E818C013F
:1089800053E0000F111F5A95E1F7880F991F080F48
:10899000191F020F131FF401848D86FD15C0F7E720
:1089A000013A1F0789F482E00E94644B81E060E095
:1089B0000E94071682E068E971E10E94CF1784EFF8
:1089C00091E00E948E1202C017FD61C08F819885D0
:1089D000801791070CF45BC01E830D8358C0198665
:1089E00045E04C838985AAE08A9FC0011124820F4B
:1089F000931F8F3F910509F008F489877B8E6A8E5B
:108A000046C0283031050CF042C02A8740C02230D1
:108A10003105ECF53B8F2A8F3AC08A81F101E80FCE
:108A2000F11D822F805D8083D7011296ED91FC911C
:108A30001397309761F182E090E0B501099527C066
:108A400080E00E94480F80E060E240E00E940A2738
:108A50001EC0D7011296ED91FC911397309721F02B
:108A600086E090E0B5010995F7018081882379F4CB
:108A700083E290E00E94412010C08C81883009F090
:108A8000E3CD80E090E0B5010E94923CDDCDC501D0
:108A90006D2D0E944C42D8CDDD248D2D6B960FB6E6
:108AA000F894DEBF0FBECDBFCF91DF911F910F9124
:108AB000FF90EF90DF90CF90BF90AF909F908F90FE
:108AC0007F906F905F904F903F902F9008951F93ED
:108AD000182F0E944B25803809F442C080E060E3E3
:108AE00072E00E94E81681E068E272E00E94E816F7
:108AF00080919E02863210F010929E0217FD04C0F3
:108B0000812F0E94D1420EC080919E020E94D142CC
:108B1000992787FD909597FF03C0909581959F4F6A
:108B200080939E0280E06CE171E00E94E81681E093
:108B300060E671E00E94E81684E068E871E00E9457
:108B4000E81685E060E971E00E94E81686E068E9D1
:108B500071E00E94E81687E060EA71E00E94E81682
:108B60001F910895DF93CF9300D000D000D0CDB7F0
:108B7000DEB7FE01319686E0DF011D928A95E9F7A6
:108B800088E089831A8284E2BF014FE759E40E949A
:108B9000882726960FB6F894DEBF0FBECDBFCF91C3
:108BA000DF910895DF93CF9300D000D000D0CDB7F0
:108BB000DEB7FE01319686E0DF011D928A95E9F766
:108BC00088E0898381E08A8384E2BF014FE759E42A
:108BD0000E94882726960FB6F894DEBF0FBECDBF41
:108BE000CF91DF910895DF92EF92FF920F931F9341
:108BF000DF93CF9300D000D000D0CDB7DEB7D82E12
:108C00008E010F5F1F4F86E0F80111928A95E9F7F8
:108C100082E089831A8287E08B838FE8E82E89E4DB
:108C2000F82E84E2B801A7010E94882781E0898399
:108C30001A82DB8284E2B801A7010E948827269667
:108C40000FB6F894DEBF0FBECDBFCF91DF911F915D
:108C50000F91FF90EF90DF900895DF93CF9300D0B6
:108C600000D000D0CDB7DEB7FE01319686E0DF013F
:108C70001D928A95E9F7198284E2BF014FE859E411
:108C80000E94882726960FB6F894DEBF0FBECDBF90
:108C9000CF91DF9108950F93DF93CF9300D000D051
:108CA00000D0CDB7DEB7542F46E14983482F4F7728
:108CB0004A83880F892F881F990B91958F778B8313
:108CC000822F8F778C83220F232F221F330B319516
:108CD00027702D83802F8F778E8307FF02C0286037
:108CE0002D83862F90E08370907024E0880F991F69
:108CF0002A95E1F79D81982B9D83552311F090646F
:108D00009D8384E2BE016F5F7F4F4FE959E40E946B
:108D1000882726960FB6F894DEBF0FBECDBFCF9141
:108D2000DF910F910895DF93CF9300D000D000D052
:108D3000CDB7DEB7FE01319696E0DF011D929A9520
:108D4000E9F794E19983982F9F779A83881F882762
:108D5000881F8B8384E2BF014FE959E40E94882772
:108D600026960FB6F894DEBF0FBECDBFCF91DF9130
:108D70000895DF93CF9300D000D000D0CDB7DEB7F9
:108D8000FE01319696E0DF011D929A95E9F78983FD
:108D9000862F8F778A83660F672F661F770B7195F3
:108DA0006F776B83842F8F778C83441F4427441FF6
:108DB0004D8384E2BF014FE959E40E94882726963B
:108DC0000FB6F894DEBF0FBECDBFCF91DF910895EF
:108DD0009C01462F83E1B9010E94B94608959C0188
:108DE000462F8DE0B9010E94B9460895DF93CF93D5
:108DF00000D000D000D0CDB7DEB7FE01319696E0AE
:108E0000DF011D929A95E9F78983862F8F778A83F0
:108E1000660F672F661F770B71956F776B8384E200
:108E2000BF014FE959E40E94882726960FB6F894AF
:108E3000DEBF0FBECDBFCF91DF910895BC0182E1AF
:108E40000E94F6460895BC018CE00E94F646089503
:108E5000DF93CF9300D000D000D0CDB7DEB7FE01B6
:108E6000319696E0DF011D929A95E9F791E1998399
:108E70008F708A83862F8F778B83661F6627661F86
:108E80006C8384E2BF014FE959E40E94882726964B
:108E90000FB6F894DEBF0FBECDBFCF91DF9108951E
:108EA000DF93CF9300D000D000D0CDB7DEB7FE0166
:108EB000319696E0DF011D929A95E9F790E199834A
:108EC0008F708A8384E2BF014FE959E40E948827AA
:108ED00026960FB6F894DEBF0FBECDBFCF91DF91BF
:108EE0000895DF93CF9300D000D000D0CDB7DEB788
:108EF000FE01319626E0DF011D922A95E9F72FE069
:108F00002983282F2F772A83880F892F881F990B71
:108F100091958F778B8367706C831D82442311F04A
:108F200081E08D8384E2BE016F5F7F4F4FE959E49A
:108F30000E94882726960FB6F894DEBF0FBECDBFDD
:108F4000CF91DF910895DF93CF9300D000D000D070
:108F5000CDB7DEB7FE01319626E0DF011D922A95DE
:108F6000E9F72EE02983282F2F772A83880F892F6E
:108F7000881F990B91958F778B8367706C8384E240
:108F8000BF014FE959E40E94882726960FB6F8944E
:108F9000DEBF0FBECDBFCF91DF910895DF93CF939A
:108FA00000D000D000D0CDB7DEB7FE01319696E0FC
:108FB000DF011D929A95E9F797E099839FE79A83DD
:108FC0009B838F778C8384E2BF0141EC59E40E943C
:108FD000882726960FB6F894DEBF0FBECDBFCF917F
:108FE000DF910895DF93CF9300D000D000D0CDB7AC
:108FF000DEB7FE01319626E0DF011D922A95E9F7E2
:1090000027E02983282F2F772A83880F892F881F0D
:10901000990B91958F778B836F776C8384E2BF0177
:1090200041EC59E40E94882726960FB6F894DEBFDB
:109030000FBECDBFCF91DF910895DF93CF9300D0C6
:1090400000D000D0CDB7DEB7FE01319626E0DF01BB
:109050001D922A95E9F727E02983282F2F772A8365
:10906000880F892F881F990B91958F778B838FE7B6
:109070008C8384E2BF0141EC59E40E948827269644
:109080000FB6F894DEBF0FBECDBFCF91DF9108952C
:10909000DF93CF9300D000D000D0CDB7DEB7FE0174
:1090A000319696E0DF011D929A95E9F7882311F435
:1090B00082E001C081E0898380E48A8384E2BE018A
:1090C0006F5F7F4F41ED59E40E94882726960FB6C7
:1090D000F894DEBF0FBECDBFCF91DF910895DF932F
:1090E000CF9300D000D000D0CDB7DEB796E0FE0120
:1090F0003196DF01292F1D922A95E9F799838F7701
:109100008A8384E2BF0141EE59E40E9488272696B3
:109110000FB6F894DEBF0FBECDBFCF91DF9108959B
:10912000DF93CF9300D000D000D0CDB7DEB7FE01E3
:10913000319696E0DF011D929A95E9F795E09983C3
:109140008F778A8384E2BF0141EE59E40E94882729
:1091500026960FB6F894DEBF0FBECDBFCF91DF913C
:109160000895DF93CF9300D000D000D0CDB7DEB705
:10917000FE01319696E0DF011D929A95E9F794E0A1
:1091800099838F778A8384E2BF0147E05AE40E9483
:10919000882726960FB6F894DEBF0FBECDBFCF91BD
:1091A000DF910895DF93CF9300D000D000D0CDB7EA
:1091B000DEB7FE01319686E0DF011D928A95E9F760
:1091C00084E089838FE78A8384E2BF0147E05AE421
:1091D0000E94882726960FB6F894DEBF0FBECDBF3B
:1091E000CF91DF910895DF93CF9300D000D000D0CE
:1091F000CDB7DEB7FE01319696E0DF011D929A955C
:10920000E9F793E0998391E09A83982F9F779B8366
:10921000881F8827881F8C8384E2BF0147E15AE4B6
:109220000E94882726960FB6F894DEBF0FBECDBFEA
:10923000CF91DF910895DF93CF9300D000D000D07D
:10924000CDB7DEB7FE01319686E0DF011D928A952B
:10925000E9F783E089831A8284E2BF0147E15AE497
:109260000E94882726960FB6F894DEBF0FBECDBFAA
:10927000CF91DF910895DF93CF9300D000D000D03D
:10928000CDB7DEB784E068EF71E00E94E81685E0B4
:1092900060E072E00E94E81689E59DE368EC70E00A
:1092A0000E944C15FE01319686E0DF011D928A95E1
:1092B000E9F78BE0898384E2BF014FE659E40E941D
:1092C0008827892B19F40E947B0EFDCF26960FB6B6
:1092D000F894DEBF0FBECDBFCF91DF910895FC01A2
:1092E0008181843219F482818B3021F0CF010E9478
:1092F000B226089580E090E00E94E82B0895FC01DA
:109300008181843219F48281883021F0CF010E945A
:10931000B226089580E090E00E94E82B0895FC01B9
:109320008181843219F48281882321F0CF010E9447
:10933000B2260895848190E00E94E82B0895FC01F4
:109340008181843219F48281853121F0CF010E941C
:10935000B2260895438150E0848190E09695982F3D
:109360008827979587956581362F3295330F330F70
:10937000307C20E0822B932B842B952B0E94E82BB2
:109380000895FC018181843219F48281873021F0B3
:10939000CF010E94B2260895858190E00E94E82BBB
:1093A0000895FC018181843219F48281882321F09F
:1093B000CF010E94B2260895838190E00E94E82B9D
:1093C0000895FC018181843219F48281853021F075
:1093D000CF010E94B2260895238130E02F773070AC
:1093E0004581942F9295990F990F907C80E0822B64
:1093F000932B248130E02F7730703695322F22273F
:1094000037952795822B932B0E94E82B0895FC011A
:109410008181843219F48281843021F0CF010E944D
:10942000B2260895838190E00E94E82B0895FC0104
:109430008181843219F48281833021F0CF010E942E
:10944000B22608958481881F8827881F9381892BDD
:1094500090E00E94E82B0895DF93CF93CDB7DEB75D
:109460002A970FB6F894DEBF0FBECDBFFE0135962A
:1094700026E0DF011D922A95E9F729E02D83282FA8
:109480002F772E83880F892F881F990B91958F77BF
:109490008F8384E2BF0148E65AE49E012F5F3F4F6D
:1094A0000E942527892B29F020E030E040E050E0A1
:1094B00004C029813A814B815C81B901CA012A9695
:1094C0000FB6F894DEBF0FBECDBFCF91DF910895E8
:1094D000DF93CF9300D000D0CDB7DEB7FC01818100
:1094E000843229F46281862F8950823020F0CF01A6
:1094F0000E94B22682C0838190E0A0E0B0E0248187
:1095000030E040E050E077E0220F331F441F551F4A
:109510007A95D1F7282B392B4A2B5B2B858190E04C
:10952000A0E0B0E07EE0880F991FAA1FBB1F7A95CC
:10953000D1F7282B392B4A2B5B2B868190E0A0E0BA
:10954000B0E075E1880F991FAA1FBB1F7A95D1F76C
:10955000282B392B4A2B5B2B878190E0A0E0B0E0D1
:109560007CE1880F991FAA1FBB1F7A95D1F7282B82
:10957000392B4A2B5B2B29833A834B835C836A30DC
:1095800059F581E060E00E9407168DB79EB70797F6
:109590000FB6F8949EBF0FBE8DBFEDB7FEB73196E4
:1095A00082E0ADB7BEB711968C938CE99CE19283B3
:1095B000818389819A81AB81BC8183839483A583D4
:1095C000B6830E9475178DB79EB707960FB6F894AD
:1095D0009EBF0FBE8DBF11C021153105410551053C
:1095E00019F080E090E002C08FEF9FEFBE016F5F47
:1095F0007F4F44E050E00E94D02B0F900F900F90CF
:109600000F90CF91DF9108951F93DF93CF9300D0F8
:1096100000D000D0CDB7DEB7182F813021F08430D4
:1096200011F08830B9F4FE01319686E0DF011D9219
:109630008A95E9F7198284E2BF0141ED59E40E945D
:10964000882740E0212F30E028233923232B29F0DD
:1096500041E003C00E943A25482F842F26960FB67A
:10966000F894DEBF0FBECDBFCF91DF911F9108955B
:10967000DF93CF9300D000D000D0CDB7DEB7982FC6
:10968000813031F0843021F0883011F0823089F45B
:10969000FE01319686E0DF011D928A95E9F782E0AE
:1096A00089839A8384E2BF0141ED59E40E948827AF
:1096B00002C00E94322626960FB6F894DEBF0FBE77
:1096C000CDBFCF91DF910895DF93CF9300D000D02D
:1096D00000D0CDB7DEB7982F813031F0843021F043
:1096E000883011F0823089F4FE01319686E0DF0186
:1096F0001D928A95E9F781E089839A8384E2BF010C
:1097000041ED59E40E94882702C00E943B2626961C
:109710000FB6F894DEBF0FBECDBFCF91DF91089595
:109720000F931F93DF93CF9300D000D000D0CDB71D
:10973000DEB78C01FE01319686E0DF011D928A952D
:10974000E9F7802F8F778983C801880F892F881FB9
:10975000990B91958F778A836F776B838FEF64E096
:10976000AF010E94F42681E060E00E94071680E0CD
:109770000E940725BC0182E00E94CF1780E090E0A4
:1097800060E040E050E00E94EF1A8FEFB8010E94C5
:10979000EF2526960FB6F894DEBF0FBECDBFCF9152
:1097A000DF911F910F910895629FD001739FF00187
:1097B000829FE00DF11D649FE00DF11D929FF00D61
:1097C000839FF00D749FF00D659FF00D9927729F98
:1097D000B00DE11DF91F639FB00DE11DF91FBD0123
:1097E000CF0111240895991B79E004C0991F9617A1
:1097F00008F0961B881F7A95C9F780950895AA1BD3
:10980000BB1B51E107C0AA1FBB1FA617B70710F06B
:10981000A61BB70B881F991F5A95A9F7809590959D
:10982000BC01CD010895FC0105900020E9F7809569
:1098300090958E0F9F1F0895FB01DC0102C00190DF
:109840000D9241505040D8F70895DC0101C06D934E
:1098500041505040E0F70895FB01DC0101900D926A
:109860000020E1F70895AEE0B0E0E9E3FCE40C94F9
:109870001B4F8C0186E08C831A8309838FEF9FE74F
:109880009E838D83CE0101960E946B4CEF81F885FB
:10989000E00FF11F10822E96E4E00C94374FAEE0FB
:1098A000B0E0E5E5FCE40C941B4F8C018EE08C836A
:1098B0001A8309838FEF9FE79E838D83CE010196E4
:1098C0000E946B4CEF81F885E00FF11F10822E96FD
:1098D000E4E00C94374FABE0B0E0E1E7FCE40C943B
:1098E0000D4F3C012B015A01FC0117821682838126
:1098F00081FD03C06FEF7FEFC6C19AE0892E1E0184
:109900000894211C311CF3012381F20123FD859170
:1099100023FF81912F01882309F4B2C1853239F4E4
:1099200023FD859123FF81912F01853229F490E059
:10993000B3010E94834EE7CF982FFF24EE24992491
:10994000FFE1FF15D0F09B3269F09C3228F4903291
:1099500059F0933291F40EC09D3249F0903369F47E
:1099600041E024C052E0F52A84E0F82A28C098E0BB
:10997000F92A25C0E0E1FE2A22C0F7FC29C0892F80
:1099800080538A3070F4F6FE05C0989C902C112408
:10999000980E15C0E89CE02C1124E80EF0E2FF2A96
:1099A0000EC09E3229F4F6FC6BC140E4F42A07C0D5
:1099B0009C3619F450E8F52A02C0983649F4F201B1
:1099C00023FD959123FF91912F01992309F0B8CFA1
:1099D000892F8554833018F08052833038F444E066
:1099E00050E0A40EB51E5FE359830FC0933631F0EB
:1099F000933779F0933509F056C020C0F501808186
:109A0000898342E050E0A40EB51E610101E010E040
:109A100012C0F501C080D180F6FC03C06FEF7FEF6C
:109A200002C0692D70E042E050E0A40EB51EC601F0
:109A30000E94784E8C015FE7F52214C0F501C080CA
:109A4000D180F6FC03C06FEF7FEF02C0692D70E09C
:109A500042E050E0A40EB51EC6010E946D4E8C017E
:109A600050E8F52AF3FE07C01AC080E290E0B30187
:109A70000E94834EEA948E2D90E008171907A8F3F0
:109A80000EC0F601F7FC8591F7FE81916F0190E021
:109A9000B3010E94834EE110EA9401501040011579
:109AA000110579F7EAC0943611F0993669F5F7FE99
:109AB00008C0F501208131814281538184E090E02A
:109AC0000AC0F501808191819C01442737FD4095B2
:109AD000542F82E090E0A80EB91E9FE6F92257FFAE
:109AE00009C050954095309521953F4F4F4F5F4F9E
:109AF000E0E8FE2ACA01B901A1012AE030E00E9493
:109B0000AF4ED82ED21840C0953729F41F2D1F7E96
:109B10002AE030E01DC01F2D197F9F3661F090377D
:109B200020F4983509F0ACC00FC0903739F0983761
:109B300009F0A6C004C028E030E00AC0106114FD9E
:109B4000146020E130E004C014FD166020E132E032
:109B500017FF08C0F501608171818281938144E023
:109B600050E008C0F50180819181BC0180E090E067
:109B700042E050E0A40EB51EA1010E94AF4ED82EC7
:109B8000D2188FE7F82EF122F6FE0BC05EEFF52219
:109B9000D91438F4F4FE07C0F2FC05C08FEEF822A9
:109BA00002C01D2D01C0192DF4FE0DC0FE01ED0DEA
:109BB000F11D8081803319F499EEF92208C01F5FEE
:109BC000F2FE05C003C08F2D867809F01F5F0F2DB0
:109BD000F3FC14C0F0FE0FC01E1510F09D2C0BC03E
:109BE0009D2C9E0C911A1E2D06C080E290E0B301C0
:109BF0000E94834E1F5F1E15C0F304C01E1510F493
:109C0000E11A01C0EE2404FF0FC080E390E0B3012D
:109C10000E94834E02FF1DC001FD03C088E790E053
:109C20000EC088E590E00BC0802F867891F001FF90
:109C300002C08BE201C080E2F7FC8DE290E0B3014C
:109C40000E94834E06C080E390E0B3010E94834EE1
:109C50009A94D914C0F3DA94F101ED0DF11D8081CD
:109C600090E0B3010E94834EDD20A9F706C080E298
:109C700090E0B3010E94834EEA94EE20C1F743CEF8
:109C8000F30166817781CB012B96E2E10C94294F99
:109C9000DC01CB01FC01E199FECF06C0FFBBEEBBAE
:109CA000E09A31960DB20D9241505040B8F70895A8
:109CB000E199FECF9FBB8EBBE09A99278DB30895A3
:109CC000262FE199FECF9FBB8EBB2DBB0FB6F8941C
:109CD000E29AE19A0FBE01960895FC010590615049
:109CE00070400110D8F7809590958E0F9F1F0895B2
:109CF000FC016150704001900110D8F7809590955B
:109D00008E0F9F1F08950F931F93CF93DF938C01A6
:109D1000EB018B8181FF1BC082FF0DC02E813F8133
:109D20008C819D812817390764F4E881F9810193BA
:109D3000F983E88306C0E885F985802F0995892B8A
:109D400031F48E819F8101969F838E8302C00FEF35
:109D50001FEFC801DF91CF911F910F910895FA0174
:109D6000AA27283051F1203181F1E8946F936E7F5A
:109D70006E5F7F4F8F4F9F4FAF4FB1E03ED0B4E04B
:109D80003CD0670F781F891F9A1FA11D680F791F8C
:109D90008A1F911DA11D6A0F711D811D911DA11D9D
:109DA00020D009F468943F912AE0269F11243019AD
:109DB000305D3193DEF6CF010895462F4770405D48
:109DC0004193B3E00FD0C9F7F6CF462F4F70405DF7
:109DD0004A3318F0495D31FD4052419302D0A9F752
:109DE000EACFB4E0A6959795879577956795BA954C
:109DF000C9F700976105710508959B01AC010A2E12
:109E000006945795479537952795BA95C9F7620FE8
:109E1000731F841F951FA01D08952F923F924F928C
:109E20005F926F927F928F929F92AF92BF92CF92EA
:109E3000DF92EF92FF920F931F93CF93DF93CDB7F3
:109E4000DEB7CA1BDB0B0FB6F894DEBF0FBECDBF6B
:109E500009942A88398848885F846E847D848C843C
:109E60009B84AA84B984C884DF80EE80FD800C8145
:109E70001B81AA81B981CE0FD11D0FB6F894DEBF28
:0C9E80000FBECDBFED010895F894FFCF98
:109E8C00FFFFFFD3282534642D2534643A200025A8
:109E9C0034640000010000FF00020000FF00070016
:109EAC0000FF0000DF41FF00030000FF00007541D0
:109EBC00FF00002441FF0000ED31FF01001C40FFBA
:109ECC000100093FFF01001C3EFF0100CC3DFF02D9
:109EDC00005A3AFF0200F23BFF0200823BFF0200F5
:109EEC00933AFF0200463AFF0200323AFF0200FEAC
:109EFC0039FF02002838FF0300CF34FF03006E3413
:109F0C00FF03040000FF03009E371B030500002223
:109F1C0003060000220300E536FF0300E036FF03D2
:109F2C00004737FF0400EA36FF0400923CFF0500AF
:109F3C00DB36FF05002F36FF0600E035FF06001A62
:109F4C0035FF06006A34FF06006634FF0700DD3279
:029F5C00FF0004
:00000001FF
